:020000040800F2
:1000000000000820BDBC00089D4C00089F4C000863
:10001000A14C0008A34C0008A54C000800000000FB
:10002000000000000000000000000000A74C0008D5
:10003000A94C000800000000AB4C0008AD4C0008C3
:100040000DBD00080DBD00080DBD00080DBD000868
:100050000DBD00080DBD00080DBD00080DBD000858
:100060000DBD00080DBD00080DBD00080DBD000848
:100070000DBD00080DBD00080DBD00080DBD000838
:100080000DBD00080DBD0008B54C00080DBD0008F1
:100090000DBD00080DBD00080DBD00080DBD000818
:1000A0000DBD0008CD4C0008014D00080DBD000835
:1000B000354D00080DBD00080DBD00080DBD000840
:1000C0000DBD00080DBD00080DBD00080DBD0008E8
:1000D0000DBD00089D5200080DBD00080DBD0008B3
:1000E0000DBD00080DBD00080DBD00080DBD0008C8
:1000F000394D00080DBD00080DBD00080DBD0008FC
:100100000DBD00080DBD0008894D00080DBD00089B
:100110000DBD00080DBD00088D4D0008C14D000843
:100120000DBD00080DBD00080DBD00080DBD000887
:100130000DBD00080DBD00080DBD00080DBD000877
:100140000DBD00080DBD00080DBD00080DBD000867
:100150000DBD00080DBD00087D5300080DBD000851
:100160000DBD00080DBD00080DBD00080DBD000847
:100170000DBD00080DBD00080DBD00080000000009
:100180000DBD00080DBD00080DBD00080DBD000827
:100190000DBD00080DBD00080DBD00080DBD000817
:1001A0000DBD00080DBD00080DBD00080DBD000807
:1001B0000DBD00080DBD00080DBD00080DBD0008F7
:1001C0000DBD00080DBD0008000000000DBD0008B9
:1001D0000DBD00080DBD00080DBD00080DBD0008D7
:1001E0000DBD00080DBD00080DBD00080DBD0008C7
:0801F0000DBD00080DBD000863
:100200000348044B834202D0034B03B118477047A5
:100210005C0000205C000020000000000548064B48
:100220001B1AD90F01EBA301491002D0034B03B1F4
:10023000184770475C0000205C00002000000000B0
:1002400010B5064C237843B9FFF7DAFF044B13B11E
:100250000448AFF300800123237010BD5C00002030
:100260000000000010BD000808B5044B1BB1044994
:100270000448AFF30080BDE80840CFE7000000006D
:100280006000002010BD00080CB410B59CB01EAB7F
:10029000029106916FF0004104910791084953F8CB
:1002A000042B0591002402A901931B9400F010F97E
:1002B000029B1C701CB0BDE8104002B0704700BF2C
:1002C0000802FFFF0EB430B59CB06FF000411FABC9
:1002D000049107910A4953F8042B029000240690D8
:1002E000084D0868019302A905951B9400F0F0F8E9
:1002F000029B1C701CB0BDE8304003B0704700BFCB
:10030000000000200802FFFF2DE9F0478F681D461E
:10031000AF420B680C46164636D8B1F90CC01CF437
:10032000906F0ED13D46184631462A4600F06EFBCE
:10033000A368DF1B2368A7602B4400202360BDE86F
:10034000F0874A69096902EB42025F1A02EBD27236
:100350006B1C52103B44934292BF914699461A46F9
:100360001CF4806F804611D0114600F071FA82466D
:1003700000B321693A4600F01BFCA38923F4906383
:1003800043F08003A38105E02F46CCE700F0BAFCE0
:10039000824658B10AEB0703A9EB0707A760C4F828
:1003A00010A0C4F8149023602F46BCE72169404692
:1003B00000F0CEFAA3890C2243F04003C8F80020D5
:1003C0004FF0FF30A381BAE72DE9F04F936817682B
:1003D00083B09246002B74D04FF0000B8B680A68F4
:1003E00081460C465D4645E0B4F90C3013F4906F3D
:1003F0002CD0D4E90401161A01EB410202EBD272AF
:10040000711C52102944914292BF904688460A4678
:100410005B0539D51146484600F01AFA01900028CC
:100420003DD03246216900F0C3FBA289019B22F432
:10043000906242F08002A2819819A8EB0606A6609D
:10044000C4F8148023612060A8462E4632465946DF
:1004500000F0DCFADAF80810A3682268A3EB0803BE
:100460003244491BA3602260CAF8081049B3D7E997
:1004700000B5083798461046002DF8D09D421E461C
:10048000B2D2A8462E46E1E70146484600F03AFCC3
:1004900003460028D0D12169484600F059FAA389C3
:1004A0000C2243F04003C9F800204FF0FF30A38135
:1004B00000220023CAF80820CAF8043003B0BDE8BF
:1004C000F08F00200023CAF8043003B0BDE8F08F9D
:1004D0002DE9F04F1C468B891D069DB0884681464C
:1004E000934603D50B69002B00F0F180002309939C
:1004F00043F22003ADF829309BF800307D4D039482
:100500000126002B73D0DA4603E01AF8013F002BD6
:1005100075D0252BF9D1BAEB0B0473D19AF80020D2
:10052000002A64D000234FF0FF32CDE905230AF101
:10053000010A049307938DF853301A9305E0049A47
:1005400006FA03F31A430492A2465446052214F80D
:10055000011B284600F0DCFAA346431B0028EED11D
:10056000049BD80644BF20228DF8532019079AF81F
:10057000001044BF2B228DF853202A2950D1039A12
:1005800011680432002903927CDB07919AF801106C
:100590002E295BD0584C0322204600F0B9FA38B11E
:1005A000049B001B4022824013430BF1010B049378
:1005B0001BF8011B51488DF82810062200F0A8FAFC
:1005C000002865D04E4B002B55D003AA00924D4B0E
:1005D000424604A94846AFF3008007467A1C06D07D
:1005E000099B3B4409939BF80030002B8BD1B8F852
:1005F0000C305B067AD409981DB0BDE8F08FBAEBD9
:100600000B04F4D023465A4641464846FFF77CFE89
:100610000130ECD0099B9AF80020234409937FE72E
:10062000A1F13002092A88BFD346B1D8079B00E068
:100630000134217803EB830302EB4303A1F1300281
:10064000092AF5D92E290793A346A3D19BF80110B7
:100650002A2927D1039B9BF802101A6805920433BC
:10066000002A0BF102000393B8BF4FF0FF3383461B
:10067000B8BF05938EE7039B073323F007030833C6
:100680000393ADE7494243F00203079104937DE7EA
:1006900003AA00921B4B424604A9484600F0F6FB11
:1006A00007469BE7A1F130020023092A05930BF1CD
:1006B000010B3FF66FAF1BF8011F03EB830302EB47
:1006C0004303A1F13002092AF5D9059362E74021DD
:1006D00000F0BEF8C8F80000C8F8100018B14023B8
:1006E000C8F8143002E70C23C9F800304FF0FF308F
:1006F00082E700BF9CBE0008A4BE0008A8BE000898
:10070000000000000903000870B50F4B0F4DAB420D
:10071000A3EB050607D0B610002455F8043B0134BE
:100720009847A642F9D80BF0F3FA094D094B5E1B26
:10073000AB424FEAA60606D0002455F8043B01342C
:100740009847A642F9D870BD18C1000818C1000822
:1007500018C100081CC10008830730B547D0541EDB
:10076000002A3ED0CAB2034601E0013C39D303F867
:10077000012B9D07F9D1032C2CD9CDB205EB052512
:100780000F2C05EB054535D9A4F1100222F00F0C12
:1007900003F1100EE6444FEA121C1A46C2E9005556
:1007A000C2E9025510327245F8D10CF1010214F081
:1007B0000C0F03EB021204F00F0C13D0ACF1040386
:1007C00023F003030433134442F8045B9342FBD148
:1007D0000CF003042CB1C9B21C4403F8011BA34262
:1007E000FBD130BD64461346002CF4D1F9E7034633
:1007F0001446C0E71A46A446E0E700BF014B18685C
:10080000704700BF0000002070B5104E33680546E9
:100810000C46B3B12146284600F07EFC431C0CD0A8
:10082000C41C24F00304A04205D0211A284600F07D
:1008300073FC013001D0204670BD4FF0FF342046DC
:1008400070BD194600F068FC3060E3E778000020D6
:100850002DE9F843CD1C25F0030508350C2D38BFD4
:100860000C25002D064618DBA94216D8DFF8DC80DF
:1008700000F04EFCD8F80420A2B1144603E06368EF
:1008800022467BB11C4623685B1BF8D40B2B1FD878
:100890009442636854D053600CE00C233360002012
:1008A000BDE8F88329463046FFF7AEFF431C0446F7
:1008B00019D00560304600F02DFC04F10B00231D1B
:1008C00020F00700C21A1CBF1B1AA350BDE8F88312
:1008D00061199442256014BF5160C8F80410635137
:1008E00063684B60E6E7D8F804701FB33C467F6846
:1008F000002FFBD123683946304604EB030900F092
:100900000BFC814516D12368ED1A29463046FFF7C6
:100910007BFF01300ED02368D8F804202B442360DD
:10092000536883B1A34203D01A465B689C42FBD153
:100930000023B0E70C233360304600F0EBFBAEE75A
:10094000C8F80430B6E7C8F80470B3E778000020B0
:10095000002950D038B551F8043C0C1F002BB8BF0B
:10096000E418054600F0D4FB274A13682BB1A342D4
:100970000CD92168601883422CD06360284614602B
:10098000BDE8384000F0C6BBA3420FD81A465B68EA
:10099000002BF9D111685018844217D02CD3636012
:1009A00054602846BDE8384000F0B4BB11685018C8
:1009B000A04214D020D8216860188342EFD1186873
:1009C0005B680844C4E900035460EAE723680B4409
:1009D0001360E6E718685B6808442060CDE720688C
:1009E0000144501883421160DBD1D3E90004014473
:1009F000C2E90014D5E770470C232B602846BDE8F8
:100A0000384000F087BB00BF7C00002088420ED930
:100A10008B1883420BD900EB020C002A6ED0624681
:100A200013F801CD02F801CD9942F9D170470F2A90
:100A30000FD8034602F1FF3C002A5FD00CF1010CF5
:100A4000013B8C4411F8012B03F8012F6145F9D1CA
:100A5000704740EA01039B0751D1A2F1100370B522
:100A600001F1200C23F00F0501F1100E00F110042C
:100A7000AC441B095EF8105C44F8105C5EF80C5C3A
:100A800044F80C5C5EF8085C44F8085C5EF8045CB2
:100A900044F8045C0EF1100EE64504F11004E9D1AF
:100AA000013312F00C0F01EB031102F00F0400EB05
:100AB000031328D0043C24F003064FEA940C1E4490
:100AC0001C1F8E465EF8045B44F8045FB442F9D103
:100AD0000CF1010402F0030203EB840301EB840137
:100AE00002F1FF3C4AB10CF1010C013B8C4411F8BE
:100AF000012B03F8012F6145F9D170BD704702F158
:100B0000FF3C03469AE72246EAE700BF00000000E8
:100B100001F0FF01102A2BDB10F0070F08D010F8AE
:100B2000013B013A8B422DD010F0070F42B3F6D1B2
:100B3000F0B441EA012141EA014122F007047FF0CB
:100B400000070023F0E80256083C85EA010586EA22
:100B5000010685FA47F5A3FA87F586FA47F6A5FA5E
:100B600087F68EB9EED1F0BC01F0FF0102F007026A
:100B700032B110F8013B013A83EA010313B1F8D115
:100B80000020704701387047002D06BF35460338F6
:100B9000073815F0010F07D1013015F4807F02BF2F
:100BA000013015F4C03F0130F0BC0138704700BF80
:100BB000844641EA000313F003036DD1403A41D368
:100BC00051F8043B40F8043B51F8043B40F8043B27
:100BD00051F8043B40F8043B51F8043B40F8043B17
:100BE00051F8043B40F8043B51F8043B40F8043B07
:100BF00051F8043B40F8043B51F8043B40F8043BF7
:100C000051F8043B40F8043B51F8043B40F8043BE6
:100C100051F8043B40F8043B51F8043B40F8043BD6
:100C200051F8043B40F8043B51F8043B40F8043BC6
:100C300051F8043B40F8043B51F8043B40F8043BB6
:100C4000403ABDD2303211D351F8043B40F8043B56
:100C500051F8043B40F8043B51F8043B40F8043B96
:100C600051F8043B40F8043B103AEDD20C3205D366
:100C700051F8043B40F8043B043AF9D2043208D05E
:100C8000D2071CBF11F8013B00F8013B01D30B88D0
:100C900003806046704700BF082A13D38B078DD0AE
:100CA00010F003038AD0C3F10403D21ADB071CBF80
:100CB00011F8013B00F8013B80D331F8023B20F8EA
:100CC000023B7BE7043AD9D3013A11F8013B00F823
:100CD000013BF9D20B7803704B7843708B788370AB
:100CE00060467047024B01461868FFF7B1BD00BF70
:100CF00000000020024B01461868FFF729BE00BF24
:100D0000000000202DE9F041144641B30AB3064625
:100D10000D4600F013FA8442074602D8B4EB500F98
:100D200013D821463046FFF793FD804650B1BC42B0
:100D30002246294628BF3A46FFF73AFF2946304661
:100D4000FFF706FE4046BDE8F081A8464046BDE8F4
:100D5000F081A046FFF7FCFD4046BDE8F081BDE80C
:100D6000F0411146FFF774BD2DE9F84F92461F463A
:100D70000A698B68DDF828909A42B8BF1A46CAF80B
:100D8000002091F843300C46064613B10132CAF8F0
:100D90000020226891065FD5DAF800300233CAF8E5
:100DA0000030226812F0060F11461DD1E168994209
:100DB000D8BF114618DD4FF0000804F1190B05E00B
:100DC000E568DAF80030ED1A45450CDD01235A4696
:100DD00039463046C847013008F10108F0D14FF0DC
:100DE000FF30BDE8F88F216894F84330003B18BF0E
:100DF00001238A060AD5E1185A1C302081F84300E5
:100E0000224494F8451082F84310023304F143025F
:100E100039463046C8470130E1D02368DAF800503F
:100E2000216903F00603042BD4E902201BD08A4277
:100E300020DD4FF00008521A90441A34002501E0DA
:100E4000454517DA0123224639463046C847013066
:100E500005F10105F4D1C2E712F0060F0DD0003BF9
:100E600018BF0123D2E7401B8A4220EAE078E2DC87
:100E70000028E2DC0020BDE8F88FE168DAF80030F5
:100E80009942D8BF114696DCAEE700BF2DE9F04786
:100E9000174684B00A7E0C9D0C460646984601F122
:100EA000430C002A35D0A2F15803D9B2202969D8C1
:100EB000202B67D8DFE813F0E600660066006600C6
:100EC0006600660066006600660066006600AC00AC
:100ED00070006600660066006600700066006600CE
:100EE0006600660021008300C60066006600B6004A
:100EF0006600830066006600EC002B68226861696A
:100F0000181D286010061B6802D4520600F1E0800C
:100F100019600023E1462361CDF800803B4603AA17
:100F200021463046FFF720FF013020D023694A4692
:100F300039463046C047013019D02368E068DDF8F3
:100F40000C909B0718D5484516DD002504F1190AB9
:100F500004E0E068A0EB0903AB420DDD012352463B
:100F600039463046C047013005F10105F1D14FF057
:100F7000FF3004B0BDE8F0874845B8BF484604B02C
:100F8000BDE8F08784F84220012004F142090023E3
:100F9000206184F84330BFE72A682368111D1806D2
:100FA000296002D4590600F1958010680146002896
:100FB0006268C0F2938054484FF00A0E15E0206832
:100FC0002B6810F0800F53F8041B02D1400648BF75
:100FD00089B26F2A4C482B6014BF4FF00A0E4FF0B5
:100FE000080E0023626884F84330002AA26051DBB7
:100FF000236823F00403236000294BD1002A7BD10E
:10100000E146BEF1080F56D0ACEB0903236183E73C
:101010002B681A6804332B6004F1420984F84220DB
:101020000120B4E72B686268191D2960D3F800908D
:1010300000214846FFF76CFD002863D0A0EB0900B3
:101040006060A4E7236843F02003236078222F48E0
:1010500084F845202A6813F0800F52F8041B03D14E
:1010600013F0400F18BF89B22A60DA0744BF43F07B
:101070002003236019B9236823F0200323604FF075
:10108000100EAEE7582384F845301F482368E1E787
:101090002368DBE77546E146B1FBF5F305FB131A60
:1010A0000A46AA4210F80A1009F8011D1946F3D29F
:1010B000BEF1080FA8D12368DD07A5D562682369B2
:1010C0009A42A1DC302309F8013C09F1FF399BE782
:1010D00019801EE7B2F90010084668E72D20002AA3
:1010E000A26084F8430002DB23F0040323600A2596
:1010F00005484942AE46CEE7037884F8423004F111
:1011000042097EE7606842E7B0BE0008C4BE00083E
:10111000704700BF704700BF38B5074D0022044636
:1011200008462A600AF09CFA431C00D038BD2B68A0
:10113000002BFBD0236038BDBC01002051F8043CDB
:10114000181F002BBCBF0B58C018704753B94AB9C1
:10115000002908BF00281CBF4FF0FF314FF0FF30BF
:1011600000F06AB9ADF1080C6DE904CE00F006F8A4
:10117000DDF804E0DDE9022304B070472DE9F04713
:10118000089D0E4604460F46002B4AD194468C45D6
:10119000B2FA82F260D942B1C2F12003974020FA3C
:1011A00003F30CFA02FC1F4394404FEA1C4E1FFA53
:1011B0008CF6B7FBFEF1230C0EFB117743EA0743D5
:1011C00001FB06F098420AD91CEB030301F1FF373B
:1011D00080F01581984240F21281023963441B1A53
:1011E000A4B2B3FBFEF00EFB103344EA034400FB51
:1011F00006F6A6420AD91CEB040400F1FF3380F086
:101200000081A64240F2FD806444023840EA014079
:10121000A41B00211DB1D4400023C5E90043BDE853
:10122000F0878B4205D90DB1C5E9000100210846C0
:10123000F5E7B3FA83F1002946D1B34202D38242E3
:1012400000F2F580841A66EB030201201746002D98
:10125000E5D0C5E90047E2E7002A40F09380A1EB22
:101260000C034FEA1C471FFA8CFE0121B3FBF7F673
:1012700007FB1630230C43EA00430EFB06F09842AE
:1012800008D91CEB030306F1FF3802D2984200F2A2
:10129000D08046461B1AA4B2B3FBF7F007FB10330D
:1012A00044EA03440EFB00FEA64508D91CEB0404E7
:1012B00000F1FF3302D2A64500F2B6801846A4EB37
:1012C0000E0440EA0640A5E7C1F120078B4022FA50
:1012D00007FC4CEA030C06FA01FE20FA07F426FA92
:1012E00007F344EA0E0400FA01F84FEA1C404FEA03
:1012F0001449B3FBF0FE1FFA8CF600FB1E3349EADB
:1013000003430EFB06F9994502FA01F20BD91CEBD7
:1013100003030EF1FF3A80F08580994540F2828008
:10132000AEF1020E6344A3EB0909A4B2B9FBF0F3DA
:1013300000FB139944EA094403FB06F6A64208D9C8
:101340001CEB040403F1FF3068D2A64266D9023BCD
:10135000644443EA0E40A41BA0FB02E6B442734679
:10136000B14652D34FD05DB1B8EB030264EB090430
:1013700004FA07F722FA01F31F43CC40C5E90074D1
:1013800000214CE7C2F1200120FA01F30CFA02FC23
:1013900026FA01F1964033434FEA1C471FFA8CFEB0
:1013A000B1FBF7F007FB1016190C41EA064100FBF0
:1013B0000EF68E4204FA02F408D91CEB010100F18A
:1013C000FF382DD28E422BD902386144891B9BB243
:1013D000B1FBF7F607FB161143EA014306FB0EF1DA
:1013E000994208D91CEB030306F1FF3814D2994245
:1013F00012D9023E63445B1A46EA004136E7394699
:10140000EDE6184602E7F045ADD2BEEB020366EB0F
:101410000C060138B146A6E74646ECE7034698E7D6
:101420004046D3E7D6467EE76444023847E708469D
:101430000DE7023E63442DE7704700BF00B500F0A2
:101440000700C0F1070CBCF1040F28BF4FF0040CDB
:10145000031D062B0FD9C31E4FF0FF3E0EFA0CF0F2
:1014600021EA000199400EFA03FE22EA0E0241EA47
:1014700002005DF804FB0023EEE70000064B074A7C
:101480001A6000225A609A60DA604FF400611961B4
:101490005A6114229A61704740050020002C0140D7
:1014A00000B583B00D4B1A6B42F480021A631B6BBC
:1014B00003F480030193019B094BD8680022114675
:1014C000C0F30220FFF7BAFF0001C0B2054B83F85A
:1014D000460340229A6003B05DF804FB00380240E6
:1014E00000ED00E000E100E082B0028802F00102BD
:1014F0001A700288C2F340025A700288C2F3800256
:101500009A700288C2F3C002DA700288C2F3001235
:101510001A710288C2F340125A710288C2F3801213
:101520009A710288C2F3C012DA710288C2F30022F3
:101530001A720288C2F340225A720288C2F38022D1
:101540009A720288C2F3C022DA720288C2F30032B1
:101550001A730288C2F340325A738278384B1A7079
:10156000828807EE902AF8EE677AC3ED017AC28886
:1015700007EE902AF8EE677AC3ED027A028907EE49
:10158000902AF8EE677AC3ED037A428907EE102AB3
:10159000B8EE477B9FED285B87EE056BFCEEC67BC4
:1015A000CDED017A9DF804201A75818907EE901A15
:1015B000F8EE677AC3ED067AC18907EE901AF8EE65
:1015C000677AC3ED077A018A07EE901AF8EE677A18
:1015D000C3ED087A418AD982818A07EE901AF8EE23
:1015E000677A9FED187A67EE877AC3ED0A7AC18A27
:1015F00007EE901AF8EE677A67EE877AC3ED097AFC
:10160000018B07EE901AF8EE677A67EE877AC3EDE2
:101610000C7A418B07EE901AF8EE677A67EE877ABC
:10162000C3ED0B7A084BA3FB0232D208074B1A60BA
:1016300002B07047AFF30080000000000000594086
:10164000C801002000008043CDCCCCCC100300208A
:101650000F4B1B6813F0400F04D00D4A136823F0A2
:10166000400313600A4B1A6822F00202104318600C
:101670001A6822F00102114319601B6813F0400F31
:1016800004D1034A136843F040031360704700BF5E
:1016900000380040B0F5805F01D340F6FF70074B83
:1016A000986029B11A461B6843F001031360704724
:1016B000024A136823F0010313607047007400406E
:1016C0000023034A1370034A1380034A13807047B0
:1016D000C4010020C2010020C001002030B40B88EA
:1016E00004881B1BD1ED017A03F6B73C41F26E74FE
:1016F000A44518D890ED027A06EE903AF8EEE66A24
:1017000027EE267A284C2468284D2D68641B06EEA7
:10171000904AF8EE666A27EE267A9FED256AC7EEB4
:10172000066A77EEA67AD0ED016A9FED227AF4EE92
:10173000C77AF1EE10FA09DC9FED1F7AF4EEC77A52
:10174000F1EE10FA04D5DFED1C7A01E0DFED197A35
:10175000C1ED017A07EE103AB8EEC77A27EE267A85
:10176000DFED166A37EE267AFDEEE77AF8EEE77AD5
:1017700077EE877AFDEEE77A17EE900AB0F57A7F7A
:1017800006DB4DF6E053984204DD4DF6E05001E0F3
:1017900042F26020022A02D080B230BC7047024B75
:1017A0001A68024B1A60F7E7200300201803002094
:1017B0000000C8420000FA460000FAC600000047D8
:1017C00038B50C46C0F30E0500210846FFF740FF70
:1017D00001224FF480412C4805F0CFFA01224FF44A
:1017E00080512A4805F0C9FA294B1B6813F0400FB5
:1017F00004D1274A136843F04003136000224FF4DA
:101800008051214805F0B9FA0023214A926812F06C
:10181000020F05D15A1CB3F57A7F01D21346F4E7C3
:101820001B4B9D8100231A4A926812F0010F05D1CB
:101830005A1CB3F57A7F01D21346F4E7144BDB68E8
:101840000023134A926812F0020F05D15A1CB3F517
:101850007A7F01D21346F4E70D4B9C8100230C4A9A
:10186000926812F0010F05D15A1CB3F57A7F01D2AC
:101870001346F4E7064BDB6801224FF4805102481F
:1018800005F07BFA38BD00BF00040240000C0240A6
:101890000038004070B506460D46002408E036F8D2
:1018A0001410054B33F81400FFF78AFF0134A4B27B
:1018B000AC42F4D370BD00BFE0BF0008F8B50F46DE
:1018C0001646012806D90546B0F5805F03D94FF4C6
:1018D000805500E00225B6F5005F01D341F6FF76A2
:1018E00004211E20FFF76CFF00242DE0012234E0CC
:1018F000012238E0A91A89B2012909D9013989B22E
:10190000ABB1A21A03FB02F292FBF1F2831A0BE0D5
:101910000121F5E7012D2ED96A1E92B23BB104FBDD
:1019200003F393FBF2F31B1A13F5005F25DBB3F50A
:10193000005F24DA99B2890089B204F5C04080B210
:10194000FFF73EFF0134A4B2A5421BD93046730015
:10195000002FDFD06A08012DC8D99442CAD2012ACB
:10196000C6D9013A92B2002BE1D004FB03F393FBFA
:10197000F2F31B1AD8E70122D0E7054BDAE741F66C
:10198000FF73D7E700211E20FFF71AFFF8BD00BF45
:1019900000E0FFFF70B50646194B187858B30D46A6
:1019A0004B1E9BB20B2B25D8164B1B880B44164A9B
:1019B0001288934220D80024AC4215D236F8143055
:1019C00003F5005292B2B2F5804F17D20D4A10883B
:1019D000204480B2990089B200F5C04080B2FFF780
:1019E000EFFE0134A4B2E7E7064B1A8815441D80C8
:1019F000012000E0002070BD0020FCE70020FAE795
:101A0000C4010020C0010020C201002000B583B045
:101A100001224FF48051164805F0AFF90022402111
:101A2000144805F0AAF90023019302E0019B013359
:101A30000193019BB3F57A7FF8D3012240210D4831
:101A400005F09BF942210C48FFF724FF00211E20DE
:101A5000FFF7B6FE01211D20FFF7B2FE01224FF471
:101A60000061064805F089F903B05DF804FB00BF8A
:101A700000040240000802405CBF0008000C024065
:101A800000B583B001224FF400610F4805F075F9ED
:101A900001211E20FFF794FE01211D20FFF790FE7B
:101AA0000023019302E0019B01330193019BB3F5F5
:101AB0007A7FF8D300224FF40061034805F05DF906
:101AC00003B05DF804FB00BF000C024008B5002124
:101AD0001E20FFF775FE01224FF40061014805F05A
:101AE0004CF908BD000C024070B5012806D9044627
:101AF000B0F5805F03D94FF4805400E0022419B19F
:101B00000F2902D90F2100E001210D0205F47065B3
:101B100045F01105264601F00F0104FB01F119B152
:101B2000B1F5803F35D20E4642211B48FFF7B2FE89
:101B3000FFF7CCFF43F230012720FFF741FE4FF4BF
:101B400000713720FFF73CFE40F201112B20FFF718
:101B500037FE29462820FFF733FEB1B22920FFF7D0
:101B60002FFE00211F20FFF72BFE00215C20FFF736
:101B700027FE00215D20FFF723FE611E89B20901C7
:101B800089B25E20FFF71CFE01211D20FFF718FE21
:101B900070BD4FF6FF76C7E7D8BE0008831E9BB224
:101BA00040F6FE72934201D90020704710B50446FA
:101BB000FFF78CFFFFF784FD01212046FFF794FF1C
:101BC00004211E20FFF7FCFD044B1C80044B002267
:101BD0001A800120034B187010BD00BFC201002005
:101BE000C0010020C401002008B5044B1B7813B9C4
:101BF000FFF766FD08BDFFF769FFF9E7C4010020A4
:101C000010B540F4004400210846FFF721FD0122F1
:101C10004FF480412C4805F0B0F801224FF4805178
:101C20002A4805F0AAF82A4B1B6813F0400F04D18C
:101C3000274A136843F04003136000224FF4805199
:101C4000214805F09AF80023214A926812F0020F09
:101C500005D15A1CB3F57A7F01D21346F4E71C4B29
:101C60009C8100231A4A926812F0010F05D15A1C78
:101C7000B3F57A7F01D21346F4E7154BDB680023F6
:101C8000134A926812F0020F05D15A1CB3F57A7FFD
:101C900001D21346F4E700230D4A93810C4A92685F
:101CA00012F0010F05D15A1CB3F57A7F01D2134609
:101CB000F4E7074BDC68A4B201224FF480510248DC
:101CC00005F05BF8204610BD00040240000C024005
:101CD000003800402DE9F04106460C4615461F46E7
:101CE000BDF81880FFF7ECFC1CB1012C02D80224CF
:101CF00003E01024B4F5805F04D835B10F2D05D969
:101D00000F2503E04FF48054F7E70125B8F5005F95
:101D100001D341F6FF7829462046FFF7E5FE42460B
:101D200039462046FFF7CAFD36B1FFF7A9FE1E204F
:101D3000FFF766FFBDE8F081FFF7C8FEF7E7F8B5EB
:101D400005460F4614461E46FFF7BAFC67B31CB1A2
:101D50003F2C02D93F2400E0012405F00305A40034
:101D6000E4B22543330103F0F00340F201141C43B5
:101D700043F212212720FFF723FD29463720FFF7E2
:101D80001FFD21462820FFF71BFDBDF81810292054
:101D9000FFF716FD00211F20FFF712FDFFF770FE71
:101DA0001E20FFF72DFFF8BDFFF790FEF8E72DE9A5
:101DB000F04F83B001900F4615461C46BDF834B075
:101DC0000020FFF71DFF82460120FFF719FF814623
:101DD0000220FFF715FF80466020FFF711FF9DF8F6
:101DE00030301B0103F0F00340F201161E431CB11A
:101DF0003F2C02D93F2400E00124BBF1000F01D1A8
:101E00004FF6FF7B05F00305A400E4B22543BAF1C9
:101E1000000F36D1012419F4F47F00D0002418F407
:101E20000E6F00D0002410F03F0F00D0002427B127
:101E3000019B13F0010F00D100242720FFF7E0FEE3
:101E400043F21223984200D000242820FFF7D8FE46
:101E5000B04200D000242920FFF7D2FE584500D020
:101E600000241F20FFF7CCFE00B100243720FFF72D
:101E7000C7FEA84200D0002484F0010003B0BDE8F2
:101E8000F08F0024C7E7000038B5054608B10023ED
:101E900003701A4B1B783BB1194B1B88012B03D9DC
:101EA000184A1288934207D0FFF79EFE1E20FFF7C4
:101EB000A7FE0446204638BD00211E20FFF780FC07
:101EC00000215D20FFF77CFC0D4B1988013989B298
:101ED000090189B25E20FFF773FC01211D20FFF785
:101EE0006FFCFFF7CDFD1E20FFF78AFE0446FFF7CB
:101EF000E7FB002DDED001232B70DBE7C4010020BF
:101F0000C2010020C00100202DE9F04F83B08346BC
:101F10000F4614461D460020FFF772FE8246012040
:101F2000FFF76EFE81460220FFF76AFE80466020C2
:101F3000FFF766FE1CB1012C02D8022403E0102436
:101F4000B4F5805F04D835B10F2D05D90F2503E016
:101F50004FF48054F7E701252E0206F4706646F030
:101F60001106019405F00F0504FB05F51DB1B5F54B
:101F7000803F4CD20195013CA4B22401A4B2BAF135
:101F8000000F48D1012519F4F47F00D0002518F482
:101F90000E6F00D0002510F03F0F00D000251FB1BC
:101FA0001BF0010F00D100252720FFF729FE43F287
:101FB0003003984200D000252820FFF721FEB042D0
:101FC00000D000252920FFF71BFEBDF80430984201
:101FD00000D000251F20FFF713FE00B100255D2073
:101FE000FFF70EFE00B100255E20FFF709FEA042BC
:101FF00000D000252B20FFF703FE40F2011398428A
:1020000000D0002585F0010003B0BDE8F08F4FF649
:10201000FF730193AFE70025B5E7000038B504462C
:1020200000210220FFF714FB1E4D01224FF48051C6
:10203000284604F0A2FE01224FF48041284604F015
:102040009CFE05F5006501224FF48051284604F0FE
:1020500094FE00224FF40051284604F08EFE002327
:10206000114A926812F0020F05D15A1CB3F57A7F1B
:1020700001D21346F4E70C4B9C8100230A4A926874
:1020800012F0010F05D15A1CB3F57A7F01D2134625
:10209000F4E7054BDB6801224FF40051034804F0DC
:1020A0006CFE38BD0004024000380040000C0240C5
:1020B0002DE9F0410546F9B94FF4005747F480780F
:1020C000C2F30D0646F48046C2F38D3242F48044DA
:1020D0004046FFF7A3FF3046FFF7A0FF2046FFF77B
:1020E0009DFF4FF44040FFF799FF05B9474638463A
:1020F000FFF794FFBDE8F08142F20207DEE700003F
:1021000010B5092813D8DFE800F00513212F3D4B47
:102110005965717D414C01224FF48061204604F0E5
:102120002CFE00224FF48061204604F026FE10BDF4
:102130003A4C01224FF40061204604F01EFE0022BA
:102140004FF40061204604F018FEF0E7334C012202
:102150004FF48051204604F010FE00224FF48051CD
:10216000204604F00AFEE2E72C4C01224FF4005115
:10217000204604F002FE00224FF40051204604F0F5
:10218000FCFDD4E7254C01224FF48041204604F0A9
:10219000F4FD00224FF48041204604F0EEFDC6E736
:1021A0001E4C01224FF40041204604F0E6FD0022BF
:1021B0004FF40041204604F0E0FDB8E7184C01223E
:1021C0001021204604F0D9FD00221021204604F001
:1021D000D4FDACE7124C01222021204604F0CDFDB5
:1021E00000222021204604F0C8FDA0E70C4C01226B
:1021F0004021204604F0C1FD00224021204604F089
:10220000BCFD94E7064C01228021204604F0B5FD78
:1022100000228021204604F0B0FD88E7001802402B
:102220000004024038B5044600224FF48041814842
:1022300004F0A3FD00224FF400717F4804F09DFDDF
:10224000002300E00133B3F5FA7FFBD301224FF402
:102250008041784804F091FD01224FF400717648E6
:1022600004F08BFD002300E00133B3F5FA7FFBD3CC
:10227000631E032B39D8DFE803F0023A6FA66D4CDA
:1022800001224FF40061204604F077FD00224FF454
:102290008061204604F071FD002300E00133B3F5B6
:1022A000FA7FFBD3654A136843F0400313600023B1
:1022B000624A926812F0010F04D1B3F57A7F01D817
:1022C0000133F5E75D490A6822F040020A6000E048
:1022D0000133B3F5FA7FFBD301224FF480615548F7
:1022E00004F04BFD554BDD68ADB2284638BD524C6D
:1022F00001224FF48061204604F03FFD002240217E
:10230000204604F03AFD002300E00133B3F5FA7FE4
:10231000FBD34B4A136843F0400313600023484A41
:10232000926812F0010F04D1B3F57A7F01D801331E
:10233000F5E743490A6822F040020A6000E00133F1
:10234000B3F5FA7FFBD3012240213B4804F015FD91
:102350003B4BDD68ADB2C8E7364C01224FF48061DB
:10236000204604F00AFD00224FF40061204604F0EC
:1023700004FD002300E00133B3F5FA7FFBD32F4ABD
:10238000136843F04003136000232C4A926812F054
:10239000010F04D1B3F57A7F01D80133F5E727495E
:1023A0000A6822F040020A6000E00133B3F5FA7FC8
:1023B000FBD301224FF400611E4804F0DEFC1F4BEA
:1023C000DD68ADB291E71C4C01224021204604F0AB
:1023D000D4FC00224FF48061204604F0CEFC0023A0
:1023E00000E00133B3F5FA7FFBD3154A136843F0DD
:1023F000400313600023124A926812F0010F04D1C7
:10240000B3F57A7F01D80133F5E70D490A6822F068
:1024100040020A6000E00133B3F5FA7FFBD30122EA
:102420004FF48061044804F0A8FC054BDD68ADB2B0
:102430005BE700BF0010024000140240003401407E
:102440000050014008B5044806F03CFB0023034A55
:102450001370034A136008BD10040020DE02002040
:10246000140300202DE9F04F8FB0002409940A9442
:102470000B940C940D94984B1A6B42F020021A6343
:102480001A6B02F020020192019A1A6B42F080024C
:102490001A631A6B02F080020292029A1A6B42F0DF
:1024A00004021A631A6B02F004020392039A1A6B75
:1024B00042F001021A631A6B02F001020492049ABC
:1024C0001A6B42F002021A631A6B02F002020592C2
:1024D000059A1A6B42F010021A631A6B02F010028E
:1024E0000692069A1A6B42F008021A631A6B02F0FF
:1024F00008020792079A1A6B42F040021A631B6B9C
:1025000003F040030893089BDFF8DC8122464FF478
:10251000C861404604F031FCDFF8D0912246B82172
:10252000484604F02AFC01224021484604F025FCDC
:10253000DFF8BCA122464B21504604F01EFC674E3A
:1025400001224FF48071304604F017FC22464FF40C
:102550004061304604F011FC01220C21304604F0A9
:102560000CFC01224FF48041304604F006FCDFF8F9
:1025700084B122464FF44F61584604F0FEFB584F99
:1025800001224FF48051384604F0F7FB01224FF44A
:102590008051584604F0F1FB22464FF4C171384691
:1025A00004F0EBFB01224FF40061384604F0E5FB38
:1025B00001224FF40051384604F0DFFB22464FF46D
:1025C0007E41484804F0D9FB182309930A94012559
:1025D0000B9509A9404604F0C7FA4FF4C863099364
:1025E0000A950B940C9409A9404604F0BDFAF02317
:1025F00009930A950B940C9409A9484604F0B4FA7F
:10260000082309930A950B9403230C9309A94846C0
:1026100004F0AAFA4B2309930A950B940C9409A988
:10262000504604F0A1FA4FF4F04309930A940B9436
:1026300009A9404604F098FA4FF4506309930A95AB
:102640000B940C9409A9304604F08EFA0C230993DC
:1026500011230A930B940C9409A9304604F084FAD0
:102660004FF4804309930A950B9403230C9309A913
:10267000304604F079FA41F6F04309930A950B9439
:102680000C9409A9584604F06FFA43F68213099393
:102690000A950B940C9409A9384604F065FA4FF496
:1026A000807309930A940B9409A9504604F05CFACC
:1026B00009950A940B9409A9384604F055FA4FF489
:1026C0007E4309930A950B940C9409A9054804F0DC
:1026D0004BFA0FB0BDE8F08F003802400010024006
:1026E000000C0240001802400014024000080240A2
:1026F000000002400004024010B588B0002403949A
:102700000494059406940794114B1A6C42F00052FD
:102710001A641A6C02F000520192019A1A6B42F08C
:1027200001021A631B6B03F001030293029B102347
:1027300003930323049303A9064804F015FA064BF8
:102740001968064A0A401A609C6008B010BD00BFB4
:10275000003802400000024000740040FAEFFFFF22
:102760002DE9F04192B02822002108A8FDF7F4FFDE
:1027700000240294039404940594069407942A4B2D
:102780005A6C42F400525A645A6C02F4005201929C
:10279000019A1A6B42F010021A631B6B03F01003CC
:1027A0000093009B4FF480530293022503954FF052
:1027B0000308CDF81080052707971C4E02A9304664
:1027C00004F047FE4FF4005302930395CDF81080B8
:1027D00005940694079702A9304604F03AFE4FF498
:1027E000806308934FF4827309934FF470630A93E4
:1027F0000B950C944FF400730D9318230E930F94C4
:102800001094072311930A4C08A9204605F09EFF57
:10281000636823F010036360636823F00803636058
:1028200012B0BDE8F08100BF003802400010024045
:10283000003401402DE9F04192B02822002108A87F
:10284000FDF78AFF002402940394049405940694EF
:1028500007942F4B1A6C42F480421A641A6C02F4EB
:1028600080420192019A1A6B42F002021A631B6BBA
:1028700003F002030093009B4FF4005302934FF0C8
:102880000208CDF80C800327049705260796214DF2
:1028900002A9284604F0DDFD4FF480430293CDF8F1
:1028A0000C80049705940694079602A9284604F024
:1028B000D0FD4FF400430293CDF80C8004970594AB
:1028C0000694079602A9284604F0C3FD08944FF425
:1028D000827309934FF470630A930B940C944FF432
:1028E00000730D9310230E930F94109407231193EC
:1028F000094C08A9204605F029FF636823F010035E
:102900006360636823F00803636012B0BDE8F08180
:102910000038024000040240003800402DE9F04138
:1029200092B02822002108A8FDF716FF0024029487
:1029300003940494059406940794294B5A6C42F42A
:1029400080125A645A6C02F480120192019A1A6B36
:1029500042F020021A631B6B03F020030093009BDC
:1029600080230293022503954FF00308CDF81080D1
:10297000052707971B4E02A9304604F06AFD4FF465
:10298000807302930395CDF8108005940694079701
:1029900002A9304604F05DFD4FF4806308934FF4C4
:1029A000827309934FF470630A930B950C944FF460
:1029B00000730D9318230E930F9410940723119313
:1029C000094C08A9204605F0C1FE636823F01003F6
:1029D0006360636823F00803636012B0BDE8F081B0
:1029E0000038024000140240005001402DE9F0413F
:1029F00092B02822002108A8FDF7AEFE0024029420
:102A000003940494059406940794294B5A6C42F459
:102A100000125A645A6C02F400120192019A1A6B65
:102A200042F001021A631B6B03F001030093009B49
:102A300020230293022503954FF00308CDF8108060
:102A4000082707971B4E0DEB0701304604F001FDE8
:102A5000802302930395CDF8108005940694079780
:102A60000DEB0701304604F0F4FC08944FF4827338
:102A700009934FF470630A930B9501230C934FF461
:102A800000730D9318230E930F9410940723119342
:102A9000094C08A9204605F059FE636823F010038D
:102AA0006360636823F00803636012B0BDE8F081DF
:102AB00000380240000002400054014010B586B0CA
:102AC0000024019402940394049405941D4B1A6C01
:102AD00042F001021A641B6C03F001030093009B97
:102AE000194BD86822462146C0F30220FEF7A6FC07
:102AF0000001C0B2154B83F81C034FF080521A60DE
:102B00004FF47A73ADF804300294114B039304949C
:102B100001A94FF0804006F0B1FC4FF080431A68E5
:102B200022F080021A6099680A4A0A409A605A683C
:102B300022F070025A609A6822F080029A6006B011
:102B400010BD00BF0038024000ED00E000E100E0F1
:102B500040D10C00F8BFFEFF10B586B000240194F0
:102B600002940394049405941C4B1A6C42F00802DE
:102B70001A641B6C03F008030093009B184BD86881
:102B800022462146C0F30220FEF758FC0001C0B2E5
:102B9000144B83F832034FF480225A6042F21073D0
:102BA000ADF8043002944FF40C73039304940E4C6C
:102BB00001A9204606F062FC236823F0800323600D
:102BC000A2680A4B1340A360636823F0700363603C
:102BD000A36823F08003A36006B010BD0038024054
:102BE00000ED00E000E100E0000C0040F8BFFEFF57
:102BF00010B586B0002401940294039404940594C3
:102C00001A4B1A6C42F020021A641B6C03F020036A
:102C10000093009B164BD86822462146C0F3022041
:102C2000FEF70CFC0001C0B2124B83F837034FF4DF
:102C300000025A6040F29733ADF8043002946323E7
:102C400003930D4C01A9204606F018FC236823F0DD
:102C500080032360636823F0700343F01003636014
:102C6000A36823F08003A36006B010BD00380240C3
:102C700000ED00E000E100E00014004010B586B077
:102C80000024019402940394049405941A4B1A6C42
:102C900042F010021A641B6C03F010030093009BB7
:102CA000164BD86822462146C0F30220FEF7C6FB29
:102CB0000001C0B2124B83F836034FF480025A6011
:102CC0004BF2AF33ADF804300294132303930D4C51
:102CD00001A9204606F0D2FB236823F0800323607D
:102CE000636823F0700343F010036360A36823F06C
:102CF0008003A36006B010BD0038024000ED00E084
:102D000000E100E0001000402DE9F8430023A34A51
:102D10001360A34A1360A34A1360A34A1360A34A33
:102D20001360A34A1370A34A1380A34A1360A34AF3
:102D30001360A34A1370A34A137005E0A24A00214E
:102D400022F8131001339BB20E2BF7D99E4B41F2A0
:102D500011121A809D4B0022DA81DA701A711A82E0
:102D60001A735A735A719A71DA72DA711A725A7244
:102D70009A725A709A701A70954D2A80954C2280DA
:102D800000226A606260AA60A260934E9C46BCE822
:102D90000F000FC6DCF800303380904E95E80F002E
:102DA00086E80F008E4D94E80F0085E80F008D4BEC
:102DB000DA6842F00102DA601A6842F001021A6031
:102DC00003F58063DA6842F00102DA601A6842F0C3
:102DD00001021A6003F51433D3F8B82022F001027F
:102DE000C3F8B8204FF00062DA604FF00072DA608A
:102DF0007D4A02F1080353E8003F43F080030832A4
:102E000042E800310029F3D1784BD3F8B82042F0E2
:102E10001002C3F8B820D3F8B82042F00402C3F877
:102E2000B8204FF00062DA604FF00072DA60704A4A
:102E3000D3F8B83003F0C003402B00F084806B4B14
:102E4000C3F8C0206B4AC3F8C42000246A4B1C603E
:102E50006A4B1C606A4E22460821304603F08DFF03
:102E600022468021304603F088FF664F22464FF409
:102E70008071384603F081FF22461021304603F06E
:102E80007CFFDFF89C8122464FF48061404603F0CE
:102E900074FF5D4D22460821284603F06EFF22464E
:102EA0000121284603F069FF22460221284603F04B
:102EB00064FF22464FF40061404603F05EFF224665
:102EC0002021304603F059FF06F5006601224FF439
:102ED0008061304603F051FFDFF848910122402124
:102EE000484603F04AFF01224FF48041304603F088
:102EF00044FF01224FF48041484603F03EFF012287
:102F00004FF48041404603F038FF0122402128461B
:102F100003F033FF01224FF48051384603F02DFFB8
:102F200001224FF48071304603F027FF21462046EE
:102F3000FEF7B0FB0121384603F018FF50B1FEF751
:102F400065FDBDE8F883294BC3F8C420294AC3F8BE
:102F5000C0207AE74FF48071284603F007FF00286D
:102F6000EDD12A4806F0B2FB294B186018B1294B65
:102F700001221A70E3E71E231A462749274806F064
:102F8000F5FB234C2060214806F0B2FB20600023B3
:102F9000084A1380064A1370E9E700BF380300208F
:102FA000200300201C030020340300202C030020F9
:102FB000E1020020DC0200208C02002088020020B8
:102FC000E0020020DF020020B802002020020020E2
:102FD000580200204802002034020020780200201D
:102FE0006802002000100040001001400064024010
:102FF000E4020020281001402803002024030020C0
:1030000000080240000C02400000024028BD0008F9
:103010009002002008030020980200202CBD000828
:1030200000040240001402402DE9F04107460E461C
:1030300090461D46002416E000220421144803F0A7
:103040009CFE14E000220821114803F096FE10E0D7
:10305000012204210E4803F090FE0FE0284603F001
:1030600093FF0134A4B2444510D2002FE4D1002EC6
:10307000E8D1284603F088FF002FE9D1002EEDD0DB
:1030800001220821024803F078FEE7E7BDE8F0815D
:103090000010024010B5002405282CD8DFE800F00D
:1030A000030812171C26154802F05CFC204610BDD0
:1030B000124C6421204602F00FFD204602F06DFD07
:1030C00080B2F4E70D4802F0E7FC2046EFE70C4839
:1030D00002F048FC2046EAE7094C6421204602F051
:1030E000FBFC204602F059FD80B2E0E7044802F004
:1030F000D3FC2046DBE72046D9E700BF0C060020C2
:10310000C405002038B504460D46032818BF012821
:1031100006D0013C032C2ED8DFE804F00D4565866F
:1031200001210220FEF794FA01224FF480514F480A
:1031300003F023FEEDE700224FF480414B4803F0FB
:103140001CFE00224A4B9B6813F0020F04D1B2F51B
:10315000FA7F01D80132F5E7454B9D810022444BAF
:103160009B6813F0010F04D1B2F5FA7F01D8013248
:10317000F5E73F4BDB6801224FF480413B4803F009
:10318000FCFD012240213B4803F0F7FD01224FF4F2
:103190008051394803F0F1FD01224FF48071374826
:1031A00003F0EBFD38BD00224021324803F0E5FD7D
:1031B0000022334B9B6813F0020F04D1B2F5FA7F63
:1031C00001D80132F5E72E4B9D8100222C4B9B68E4
:1031D00013F0010F04D1B2F5FA7F01D80132F5E7FF
:1031E000274BDB68C7E700224FF48051224803F0E9
:1031F000C4FD00221E4B9B6813F0020F04D1B2F5F0
:10320000FA7F01D80132F5E7194B9D810022184B56
:103210009B6813F0010F04D1B2F5FA7F01D8013297
:10322000F5E7134BDB68A6E700224FF480711348E3
:1032300003F0A3FD0022124B9B6813F0020F04D190
:10324000B2F5FA7F01D80132F5E70D4B9D810022DE
:103250000B4B9B6813F0010F04D1B2F5FA7F01D834
:103260000132F5E7064BDB6885E700BF000402404A
:103270000038004000000240000C024000100240F4
:10328000005401402DE9F84305460F4616461C46FA
:10329000AF4B00221A600121AE4803F067FD002801
:1032A00000F0D2802B8803F0010323702B88C3F336
:1032B000400363702B88C3F38003A3702B88C3F390
:1032C000C003E3702B88C3F3001323712B88C3F36F
:1032D000401363712B88C3F38013A3712B88C3F34E
:1032E000C013E3712B88C3F3002323722B88C3F32D
:1032F000402363722B88C3F38023A3722B88C3F30C
:10330000C023E3722B88C3F3003323732B88C3F3EA
:10331000403363736B883B80AB8833806B89E38178
:10332000AB8907EE903AF8EE677A9FED8B7A67EEFD
:10333000877AC7ED017AEB8907EE903AF8EE677A63
:1033400067EE877AC7ED027A2B8A07EE903AF8EE9D
:10335000677A67EE877AC6ED017A6B8A07EE903A54
:10336000F8EE677A67EE877AC6ED027AAA8A7B4B17
:103370005A83EB8ABB812B8BB3816378002B00F0DF
:10338000958001220821764803F0F7FCA378002BF2
:1033900000F0928001228021714803F0EEFCE37876
:1033A000002B00F08F8001224FF48071694803F0F8
:1033B000E4FC2379002B00F08C8001221021684866
:1033C00003F0DBFC6379002B00F0898001224FF4CD
:1033D0008061644803F0D1FCA379002B00F0868063
:1033E00001220821604803F0C8FC637A1BB1E3792D
:1033F000002B40F08180002201215B4803F0BDFCDE
:1034000000224FF40061574803F0B7FCA37A1BB1C8
:10341000237A002B40F0868000220221524803F0DC
:10342000ACFC002220214E4803F0A7FC237B1BB9F3
:103430004E4B7B604E4BBB60637B1BB94B4B736049
:103440004B4BB360BDE8F8834FF48071464803F0FE
:103450008DFC01287FF426AF464806F037F93C4B37
:10346000186000287FF41EAFDFF80C91484606F084
:1034700043FADFF8DC80C8F80000484606F01AFA84
:10348000C8F800001E222946484606F041F9C8F84F
:1034900000001E222946484606F070FAC8F80000CF
:1034A000344806F025F9C8F80000FBE600220821A0
:1034B0002B4803F062FC69E700228021284803F0D2
:1034C0005CFC6CE700224FF48071224803F055FC4D
:1034D0006FE700221021224803F04FFC72E7002220
:1034E0004FF480611F4803F048FC75E70022082173
:1034F0001D4803F042FC78E747F6FF710320FFF711
:1035000001FE47F6FF710320FFF7FCFD01224FF497
:103510000061144803F031FC01221146124803F007
:103520002CFC73E747F6FF710420FFF7EBFD47F62D
:10353000FF710420FFF7E6FD01222021084803F077
:103540001CFC01220221084803F017FC6EE700BFB3
:1035500090020020000C02400000803BB8020020D6
:103560000008024000040240000002400000204128
:103570000AD7233C28BD00082CBD000884460088DB
:10358000012304E03CF81320504001331BB28B426E
:10359000F8DB704710B50E4B1B8841F211129342B5
:1035A00005D047F2777293420FD10E2400E00D242C
:1035B0002146FFF7E3FF074B1880074B33F8143021
:1035C000984214BF0020012010BD0020FCE700BF7E
:1035D000DA020020D80200209802002010B504462C
:1035E00001210A4803F0C2FB08B1012010BD0848C0
:1035F00006F06CF808B10120F8E71E2221460548C4
:1036000006F0BCF9024806F073F8EFE7000C024040
:1036100028BD000838BD000838B5044601210D4812
:1036200003F0A4FB08B1012038BD0B4806F04EF8AA
:1036300008B10120F8E7094D2B681E2221460848F1
:1036400006F094F82B681E332B60034806F050F800
:10365000EAE700BF000C024028BD00088C020020F1
:1036600038BD000810B501210B4803F07FFB08B1FD
:10367000012010BD094806F029F808B10120F8E73B
:10368000074C204606F038F9204606F013F90348A7
:1036900006F02EF8EDE700BF000C024028BD000840
:1036A00038BD00088C4600220CE033B9074BDB69BB
:1036B00013F08003F9D00123F7E7815C034B996293
:1036C000013292B26245F1D3704700BF0010014051
:1036D0000D4B1B78002BFBD10C4BD3F8B82022F0FC
:1036E0000102C3F8B820D3F8BC206FF30F021043D7
:1036F000C3F8BC00D3F8B82042F00102C3F8B820E8
:10370000014B01221A707047E00200200064024061
:1037100072B6FEE700B585B00023009301930293D3
:1037200003932B482B4A02604FF44032426083607F
:1037300001220261836180F82030C36226498162E0
:10374000C3600521C16180F83030426102F0DEF8CB
:10375000002831D109230093012301930723029309
:1037600069461B4802F0BAFA40BB082300930223C3
:1037700001936946164802F0B1FA08BB0223009390
:10378000032301936946124802F0A8FAD0B90A232C
:1037900000930423019369460D4802F09FFA98B9FB
:1037A0000B230093052301936946094802F096FA1A
:1037B00060B905B05DF804FBFFF7AAFFFFF7A8FFAB
:1037C000FFF7A6FFFFF7A4FFFFF7A2FFFFF7A0FF99
:1037D0000C060020002001400100000F00B585B05C
:1037E000002300930193029303931448144A026048
:1037F0004FF44032426083600361836180F820307F
:10380000C362104A8262C3600122C26180F8303014
:10381000426102F07BF868B90F2300930123019302
:10382000072302936946054802F058FA20B905B00B
:103830005DF804FBFFF76CFFFFF76AFFC40500208B
:10384000002201400100000F2DE9F041B4B0002139
:103850002D912E912F913091319132913391279169
:10386000289129912A912B912C91902203A8FCF761
:1038700073FF4023039303A802F076FE002840F074
:103880009E80504B5A6C42F010025A645A6C02F0FF
:1038900010020292029A1A6B42F001021A631B6B29
:1038A00003F001030193019B4FF4007327934FF042
:1038B0000208CDF8A0800327299700242A942B948E
:1038C00007262C96404D27A9284603F0C2FD4FF449
:1038D00080632793CDF8A08029972A942B942C9667
:1038E00027A9284603F0B5FD384BD3F8B82022F0BD
:1038F000F05242F00062C3F8B820D3F8B82022F0AA
:10390000C00242F04002C3F8B820D3F8B82042F415
:103910004032C3F8B820D3F8B82022F49072C3F82C
:10392000B820D3F8B82022F40072C3F8B820D3F836
:10393000B82042F48062C3F8B820D3F8B82022F44B
:10394000C052C3F8B820D3F8B82022F4C042C3F85C
:10395000B820D3F8CC2022F00402C3F8CC201C4BB2
:10396000D86822462146C0F30220FDF767FD00011A
:10397000C0B2184B83F8250320225A604FF4E1337C
:103980002D932E942F9430940C23319332943394AE
:1039900004F1804404F588342DA9204605F00EFE7C
:1039A000636823F490436360A36823F02A03A36051
:1039B000236843F00103236034B0BDE8F081FFF7D2
:1039C000A7FE00BF00380240000002400064024031
:1039D00000ED00E000E100E008B50848084B036096
:1039E000B7234360002383600922C26003618361BF
:1039F00005F0D4F900B908BDFFF78AFE10040020D5
:103A00000044014008B50B480B4B03604FF4E13311
:103A1000436000238360C36003610C2242618361C1
:103A2000C3610362436208F018F900B908BDFFF7EB
:103A30006FFE00BF3C030020007C004000B589B051
:103A40000023049305930693079301930293039332
:103A50001348144A0260436083605B22C2600361C2
:103A60004361836105F09AF998B94FF48053049348
:103A700004A90B4805F0D4FA68B900230193029316
:103A8000039301A9064805F05DFC30B909B05DF863
:103A900004FBFFF73DFEFFF73BFEFFF739FE00BFDB
:103AA000A80400200004014000B589B00023019360
:103AB0000293039304930593069307931448154ABE
:103AC00002600122426083605B22C2600361802346
:103AD000836105F063F9A8B90D4805F08FF998B92D
:103AE000602301935B23029300220392059201A9B4
:103AF000074805F0EBF948B9054801F0C5FD09B0E4
:103B00005DF804FBFFF704FEFFF702FEFFF700FE7F
:103B1000C40300200048014000B58FB000230A9381
:103B20000B930C930D9307930893099300930193C0
:103B3000029303930493059306931E481E4A026062
:103B4000436083602D22C2600361836105F026F922
:103B500030BB4FF480530A930AA9164805F060FA67
:103B600000BB144805F04AF9F0B900230793099304
:103B700007A9104805F0E6FBC0B96023009316239F
:103B8000019300230293049308226946094805F033
:103B90009DF968B9074801F077FD0FB05DF804FBA7
:103BA000FFF7B6FDFFF7B4FDFFF7B2FDFFF7B0FD7D
:103BB000FFF7AEFDF40400200008004010B596B0F9
:103BC000002412941394149415940B940C940D9453
:103BD0000E940F94109411942C2221466846FCF701
:103BE000BBFD2548254B0360446084600823C36007
:103BF00004614461846105F0D1F8002832D14FF4AA
:103C00008053129312A91C4805F00AFA00282BD100
:103C1000194805F0F3F848BB60230B9304230C9379
:103C200000220D920F920BA9134805F04FF9F8B935
:103C30000023009301930293039304934FF40052E3
:103C40000592069307934FF00072089209930A9326
:103C50006946094805F0C6FB60B9074801F014FD44
:103C600016B010BDFFF754FDFFF752FDFFF750FDF2
:103C7000FFF74EFDFFF74CFD5C0400200000014003
:103C800000B595B03422002107A8FCF765FD00239C
:103C900002930393049305930693244B1A6C42F00A
:103CA00080521A641B6C03F080530093009B204BDE
:103CB0001A6842F440421A601B6803F440430193BF
:103CC000019B012307934FF48033089302230D9344
:103CD0004FF480020E9219220F924FF4B872109294
:103CE000119308221292139307A802F0EBF8B0B9CF
:103CF00003F052F8A8B90F23029302230393002381
:103D000004934FF4A05305934FF480530693062178
:103D100002A802F04DFB30B915B05DF804FBFFF7C7
:103D2000F7FCFFF7F5FCFFF7F3FC00BF003802409B
:103D3000007000402DE9F04387B003F007F9FFF76A
:103D40009FFFFEF78FFBFDF7ABFBFEF709FD00F0D1
:103D500089FFFEF7B3FEFEF7FFFEFFF7DBFCFFF780
:103D60003DFDFEF767FDFEF7D9FDFEF73FFEFFF7CD
:103D70006BFDFDF783FBFEF73BFFFEF77FFFFFF7D1
:103D80002BFEFFF73FFEFFF759FEFFF78DFEFFF713
:103D9000C3FEFFF713FFFEF7AFFCFEF7B5FF8D4A3A
:103DA0003523D362D36A01335B08013BD363D36A03
:103DB0009B00033302F5A032D362D36A01335B0860
:103DC000013B53630021844805F0BAF94CE0834B72
:103DD0001B78002B4FD1824A52E8003F43F4807396
:103DE00042E800310029F6D17D4A52E8003F43F015
:103DF000200342E800310029F6D1794A02F1080394
:103E000053E8003F43F00103083242E80031002943
:103E1000F3D1744B002283F8252320225A606F4B84
:103E200001221A7027E0704B00221A706F4B5A68FB
:103E30001A61FEF707FB6E4B1B78022B00F0C08562
:103E4000032B00F0F385012B09D16A4C0221204697
:103E5000FFF728FC002323706370654A1370664BDC
:103E60001B78012B00F0E4854FF48071634802F069
:103E70007DFF0128ABD0624B1B780F2BDBD801A252
:103E800052F823F0273E0008C53E00082F3F0008E7
:103E9000693F0008993F0008A93F0008C53F000896
:103EA0002D400008BD44000803450008814100087A
:103EB0005D420008AD420008634300089F430008CC
:103EC0006B4400084F4C0D212046FFF757FB4E4B2B
:103ED00018802046FFF75EFB70B9464A137843F01E
:103EE00004031370464B02221A703F4B00221A70D3
:103EF0003F4B01221A709EE7444A136843F0400387
:103F0000136002F58E32136843F040031360404B98
:103F1000404A41492046FFF7B5F9404B1A68404BEB
:103F20001A600723364A13702F4A1370E0E72F4BAD
:103F30005A681A61FEF786FAFEF7E6FEFDF754FEB0
:103F4000324A136823F04003136002F58E3213687F
:103F500023F0400313600023294A1370224A137090
:103F6000234B01221A7066E72E48FFF755FB82B2F9
:103F70002D4B1A801F490B7803430B7042B91C4B21
:103F800003221A700023184A13701D4A137052E757
:103F9000174B01221A70F5E7154B02221A70124BCB
:103FA0001A78174B1A7046E7FFF75CFB114A137833
:103FB000034313700E4B01221A700B4B1A78104BEF
:103FC0001A7038E70A4B01221A70074B1A780C4B0B
:103FD0001A7030E7000800405C040020DF02002077
:103FE0000010014000E100E007030020C8010020AC
:103FF0000603002004030020E1020020000002402C
:104000000803002098020020D80200200038004059
:1040100034020020680200207802002038030020CB
:1040200034030020B8020020D6020020B24B5A68A8
:104030001A61FEF707FAB14B1B68B14A1268934246
:104040007FF6F9AEAE4A13600120FEF7EBF8AD4FF4
:1040500038810120FEF7E6F838810220FEF7E2F809
:10406000A94E30810220FEF7DDF830810320FEF7F3
:10407000D9F80320FEF7D6F838800420FEF7D2F8EE
:104080000420FEF7CFF83080DFF8AC8201223946F9
:104090004046FDF723FB01469C4D28800320FFF797
:1040A00031F8DFF89892022231464846FDF716FBB8
:1040B000014628800420FFF725F83B89944C638053
:1040C0003389A380B8F80C100120FFF71BF8B9F86A
:1040D0000C100220FFF716F80020FEF7DBFF288007
:1040E0000120FEF7D7FF2880E0810120FEF7D2FFF4
:1040F000288020820120FEF7CDFF288060820120E9
:10410000FEF7C8FF2880A0820120FEF7C3FF2880A9
:10411000E0820220FEF7BEFF28800320FEF7BAFFF0
:1041200028800420FEF7B6FF288020830520FEF7B4
:10413000B1FF2880774B1B68774A1360E3801B0C24
:1041400023813B8863813388A381744BDB7A012B05
:1041500003D0734B07221A706DE602340D212046FE
:10416000FFF70CFA03466F4A1080A01E8383FFF707
:1041700035FA034628806C490A7813430B70E8E748
:104180006A4C03212046FFF7F9F9E38898420CD0E6
:10419000654A137843F004031370654B01221A70CB
:1041A0005F4B1A78634B1A7045E623886188A488B0
:1041B00003F00106C3F3400513F0040F1FD013F002
:1041C000080F1AD104F00F070C4641F6FF71009159
:1041D0002B463A4621463046FDF77CFD524B58703F
:1041E0003B4622463146FDF78FFE0028D5D04E4A89
:1041F000137863F07F031370CFE70127E7E705B17A
:104200000225CFB2C1F30328214309D01FB13F2FAC
:1042100002D93F2700E001273CB94FF6FF7404E0C4
:104220004FF6FF744FF002080127009443463A46C8
:1042300031462846FDF783FD3B4B58700194CDF87D
:1042400000803B462A463146FDF7B1FD0028A4D048
:10425000354A137863F07F0313709EE7324B0022D8
:104260005A70324C03212046FFF788F9E3889842C0
:104270000CD02D4A137843F0040313702C4B012209
:104280001A70274B1A782B4B1A70D4E52088638854
:10429000C3F30D03A288C2F30D0243EA8232C0F3D6
:1042A000400100F00100FDF703FFE7E71F4C032189
:1042B0002046FFF763F9E38898420CD01A4A137836
:1042C00043F0040313701A4B01221A70144B1A782E
:1042D000184B1A70AFE5234624885A889B88C4F38C
:1042E000400104F001000C422AD00F4A137843F039
:1042F00004031370E7E700BFC8010020200300207B
:104300001C0300201402002008020020D602002016
:10431000B8020020380300203003002034020020BF
:1043200007030020D8020020040300209802002088
:104330000603002008030020780200206802002005
:104340001AB1402A02D9402200E001222BB1B3F574
:10435000FA7F03D94FF4FA7300E00223FEF764FEFC
:10436000B1E77C4C03212046FFF708F9E388984227
:104370000CD0794A137843F004031370774B012271
:104380001A70774B1A78774B1A7054E56088217849
:1043900001F00101C0F30B00FDF77CF9EEE76E4B75
:1043A00000225A706B4C03212046FFF7E7F8E388A0
:1043B00098420CD0684A137843F004031370674B9B
:1043C00001221A70664B1A78664B1A7033E5228800
:1043D0006088A388022A10D0032A34D0012A3CD155
:1043E0001BB9FDF7DBFB0028E9D1FDF7FDFB5A4ABD
:1043F000137863F07F031370E1E75B4A14880022AF
:104400008DF81720184307D0FDF7EEFB524A1378BA
:1044100063F07F031370D2E70DF11700FDF734FD51
:104420004D4B58709DF817302BB94B4A137863F0F9
:104430007F031370C3E7012322461946FDF764FD8D
:104440000028BCD0F1E7184304D0434A137863F046
:104450007F031370FDF7C8FBB1E7FDF7C5FB3E4ACC
:10446000137863F07F031370A9E73B4B00225A7067
:10447000384C0D212046FFF781F8638B98420ED00F
:10448000FDF7B2FB344A137843F004031370334B47
:1044900001221A70324B1A78324B1A70CBE4204644
:1044A00030F8021BFDF776FA0028F0D1FDF79CFBEF
:1044B000294A137863F07F031370E8E72548FFF774
:1044C00069F870B9244A137843F004031370254B3C
:1044D00002221A70224B00221A70204B01221A70FD
:1044E000A9E4224B224A23491A48FCF7FDFF224B3C
:1044F0001A68224B1A6009231A4A1370184A13705B
:10450000EBE71F4B1B78012B4AD0022B00F02D81CB
:104510001C4B1B681C4A1268934200F2FE811B4B25
:104520001B78002BFBD0FDF78DFF154BDB8A032B8F
:104530000BD9174B1A68174BDA60114B1B7D164AC3
:10454000A2FB0323DB08154A1360054B09221A70EE
:1045500071E400BF9802002004030020060300203D
:104560000703002008030020C201002034020020BD
:104570006802002078020020380300203403002065
:10458000C8010020200300201C030020DE020020C0
:104590000C03002010040020CDCCCCCC1003002054
:1045A000AD4BD3ED077AFCEEE77A17EE903A99B26D
:1045B0000220FEF7A7FD0320FDF734FE0320FDF7E0
:1045C00031FEA64C20800420FDF72CFE0420FDF7D0
:1045D00029FEA34D288001222146A248FDF77EF83E
:1045E0000146A14C20800320FEF78CFD02222946C3
:1045F0009E48FDF773F8014620800420FEF782FDF7
:104600009B4C01228021204602F0B7FB0022802132
:10461000204602F0B2FB974804F00CFA002875D14E
:104620008D4B93ED027AD3ED047A37EE677AD3EDB2
:10463000036AC7EE267AB2EE047A67EE877AFCEE5A
:10464000E77ACDED037A9DF80C60DFF854920021F3
:10465000484604F021FEDFF84C820821404604F071
:104660001BFE854F3B6823F008033B60834D2B689E
:1046700023F008032B6000247C626C6221464846CC
:1046800004F05EFD0821404604F05AFDEB6A143B3D
:104690006B627C622546704BD3ED047A93ED027A0F
:1046A000F4EEC77AF1EE10FA37D5754B1B78002B74
:1046B000F1D0FCEEE77A17EE903A99B20120FEF7BE
:1046C00021FD654BD3ED047A93ED037A77EE877A7B
:1046D000C3ED047A00276B4B1F60694B1F70DFF836
:1046E000C88101224FF40071404602F046FB3A4671
:1046F0004FF40071404602F040FBB4FBF6F306FBBA
:1047000013439BB21BB10134A4B2C4E7FEE7E8B285
:10471000FDF7F6FC0135ADB2F5E7574AD36843F033
:104720000103D360FDF78EFE4B4CD4ED017AC4ED4E
:10473000047AFCEEE77A17EE903A99B20120FEF780
:10474000E1FCE38A032B0CD94A4AD0684E49086041
:1047500042F20F71D160013B642202FB03F34B4A2A
:104760001360444804F066F9D2E63B4BD3ED077A78
:10477000FCEEE77A17EE903A99B20120FEF7C2FC00
:104780000320FDF74FFD0320FDF74CFD334C208047
:104790000420FDF747FD0420FDF744FD304D28803F
:1047A000012221462F48FCF799FF01462E4C20801C
:1047B0000320FEF7A7FC022229462C48FCF78EFFB7
:1047C000014620800420FEF79DFC314B02221A7026
:1047D00000229A721A814FF47A721A812D4A5A6015
:1047E00080225A802C4B42F21072DA622B4804F07D
:1047F00021F978BB012280211D4802F0BEFA42F265
:104800001073013BFDD100228021194802F0B5FA56
:104810001F4B02229A72174804F00CF9D8B90E4BBC
:10482000D3ED047A93ED027AF4EEC77AF1EE10FA42
:104830003CD5134B1B78002BF1D0074B93ED037A3B
:1048400077EE277AC3ED047A00230E4A13600C4AF0
:104850001370E4E7FEE7FEE7C80100201402002021
:104860000802002078020020D60200206802002002
:10487000000C0240100400200048014000080040E5
:10488000DE020020140300200C030020100300208F
:10489000FC0100200004024000040140A8040020A4
:1048A000C4030020F4040020001802406C4804F007
:1048B000ACF86C4C01228021204602F05EFA002206
:1048C0008021204602F059FA674804F0FBF8674B54
:1048D00000225A62FDF7B6FD654CD4ED017AC4EDB5
:1048E000047AFCEEE77A17EE903A99B20220FEF7CE
:1048F00009FCE38A032B0CD9594AD0685D4908604A
:1049000042F20F71D160013B642202FB03F35A4A69
:104910001360534804F08EF8FAE5584A13600120FA
:10492000FDF780FC564E30810120FDF77BFC308185
:104930000220FDF777FC534F38810220FDF772FC0F
:1049400038813389504C6380A0800020FEF7A2FBA1
:104950004E4D28800120FEF79DFB2880E08101203C
:10496000FEF798FB288020820120FEF793FB288029
:1049700060820120FEF78EFB2880A0820120FEF7D6
:1049800089FB2880E0820220FEF784FB2880032038
:10499000FEF780FB28800420FEF77CFB2880208324
:1049A0000520FEF777FB2880394B1B68394A1360D6
:1049B000E3801B0C2381338863813B88A381AEE5B0
:1049C000354C0D212046FEF7D9FD344B188060830D
:1049D00000230BE02C4A32F813205900304800F82D
:1049E00013200131120A425401339BB20E2BF1D92C
:1049F0001E20FEF76DFE2B4B00221A70FFF72FBA18
:104A0000214A32F813205900254800F813200131BB
:104A1000120A425401339BB20E2BF1D91E20FEF72D
:104A200057FE204B00221A70FFF719BA0023F3E754
:104A3000174B1B681C4A12689B1A642B7FF614AA3A
:104A400000221A4B1A801A490B7843F002030B70AC
:104A5000144B01211970174B1A70FFF705BA00BFEC
:104A600010040020000C0240A804002000040140B3
:104A7000C80100200C030020100300201C030020AC
:104A80001402002008020020B8020020D6020020F4
:104A90003803002030030020BA020020D802002092
:104AA000E4020020060300202C030020DC0200208A
:104AB00004030020E102002000B583B000931346F8
:104AC0000A460146034803F0CDF900B1012003B0C6
:104AD0005DF804FB4005002000B583B00093134649
:104AE0000A460146034803F0E1FA00B1012003B091
:104AF0005DF804FB4005002008B5034803F014FEF0
:104B0000043818BF012008BD4005002008B5014643
:104B1000014803F096FD08BD4005002000B583B0B4
:104B200001238DF8073000F0ADF810B900238DF89F
:104B300007309DF8070003B05DF804FB38B5FFF7B8
:104B4000EDFF012802D00225284638BD044607485B
:104B500003F05CFD05460028F6D14FF400610348E0
:104B600003F082FD0028EFD02546EDE74005002048
:104B700008B5074B01221A70FFF7BEFF20B9044A9F
:104B8000137803F0FE031370014B187808BD00BFC3
:104B90005000002010B50446074B01221A70FFF7A1
:104BA000CDFF10B1044B187810BD2046FFF7E0FF91
:104BB000014B1870F6E700BF5000002008B5FFF762
:104BC000D7FF08BD08B5084611461A464FF0FF3317
:104BD000FFF772FF30B9FFF78FFF03460028FAD1C5
:104BE000184608BD0123FBE708B5084611461A46DA
:104BF0004FF0FF33FFF770FF30B9FFF77DFF03463B
:104C00000028FAD1184608BD0123FBE730B589B06A
:104C1000134B187810F001041BD1154603291CD83A
:104C2000DFE801F002040A100C4613E06846FFF7C3
:104C30006DFF069B2B600DE06846FFF767FF079B43
:104C40002B8007E06846FFF761FF079B5B0A2B603C
:104C500000E00324204609B030BD0424FAE700BF79
:104C60005000002008B50349034806F0F3FC034B4D
:104C7000187008BD5406002064C0000858060020C3
:104C80000020704708B50121034802F06FF808B909
:104C9000012008BD0020FCE7000C0240FEE7FEE713
:104CA000FEE7FEE7FEE770477047704708B502F081
:104CB00059F908BD08B5034800F075FF024800F037
:104CC00072FF08BD0C060020C405002008B5084A84
:104CD000136801331360074A1268934203D00648F1
:104CE00003F00FFF08BD054B01221A70F7E700BF64
:104CF000140300201003002010040020DE02002016
:104D000008B5094B1A6842F008021A6007490A6898
:104D100042F008020A60DA6822F00102DA60044810
:104D200003F0EFFE08BD00BF00480140000800404E
:104D3000C40300207047000010B5114B9B7A022B72
:104D40000ED0032B18D100210220FEF7DBF90C4C0A
:104D500000226188606802F010F80223A3720BE061
:104D6000074C21890220FEF7CDF901226188606895
:104D700002F003F80323A372024803F0C2FE10BD41
:104D8000FC010020A80400207047000008B5094B72
:104D90001B6913F0010F0BD0064B6FF001021A6173
:104DA000054A1368013313600221044801F0EBFF48
:104DB00008BD00BF0010004038030020000C024076
:104DC000064B1B6913F0010F07D0044B6FF0010273
:104DD0001A61034A136801331360704700140040DE
:104DE0002003002010B49A4B5A6AD2B2994B1A7021
:104DF000994B1B881F2B00F22B82DFE813F0200059
:104E00002F00290229022902290229022902290246
:104E1000C70029022902290229022902290229029E
:104E2000290229022902290229022902290229022A
:104E3000290229022902290296012902EF01874944
:104E400008688749086087490120087086490A80F8
:104E50000344814A13805DF8044B704782490B88F4
:104E600003EB02239BB20B8047F2777293426BD025
:104E700014D94BF6BB32934272D035D849F6991209
:104E8000934265D04AF6AA22934265D048F688023A
:104E900093426DD1704B02221A80DCE744F2444207
:104EA00093423FD00FD842F22222934228D043F2BD
:104EB000333293422DD041F21112934258D1664BB6
:104EC00002221A80C7E745F25552934233D046F288
:104ED000666293424CD100235F4A1380614A13708B
:104EE000624B06221A70B6E74CF6CC4293423BD096
:104EF0004DF6DD5293423BD1574B02221A80AAE76E
:104F00000023554A1380574A1370584B02221A70D7
:104F1000A1E70023504A1380524A1370534B0322D7
:104F20001A7098E700234C4A13804E4A13704F4B77
:104F300004221A708FE70023474A1380494A1370EE
:104F40004A4B05221A7086E7434B02221A8082E7F9
:104F5000414B02221A807EE73F4B02221A807AE7F9
:104F60003D4B02221A8076E73B4B02221A8072E701
:104F70000023394A13803B4A13703D4A137843F0AB
:104F800002031370394B02221A7064E7364909880C
:104F900048F68800814225D049F6991081423CD0DC
:104FA0004AF6AA20814269D04BF6BB30814200F01C
:104FB00080804CF6CC40814200F0968013F0010FC7
:104FC00000F0AD80590801392A4C34F8110000EB8B
:104FD000022224F8112001331F4A1380264B00229D
:104FE0001A7038E713F0010F11D05B08013B21481C
:104FF00030F8131001EB022220F813201B4B0A2279
:105000001A700023144A1380164A137023E75B08B2
:10501000013B184921F81320F0E713F0010F11D0DC
:105020005B08013B134830F8131001EB022220F813
:1050300013200E4B0B221A700023074A1380094AD3
:10504000137008E75B08013B0A4921F81320F0E7D9
:105050000010014009030020DC020020380300207A
:105060002C030020E1020020DA02002008030020C7
:1050700004030020980200200603002013F0010F13
:1050800011D05B08013B7F4830F8131001EB02227E
:1050900020F813207C4B0C221A7000237B4A1380CB
:1050A0007B4A1370D7E65B08013B764921F8132051
:1050B000F0E713F0010F11D05B08013B714830F8A5
:1050C000131001EB022220F813206F4B0D221A70EF
:1050D00000236E4A13806E4A1370BCE65B08013BE6
:1050E000684921F81320F0E713F0010F11D05B0895
:1050F000013B644830F8131001EB022220F8132022
:10510000614B0E221A700023604A1380604A1370AC
:10511000A1E65B08013B5B4921F81320F0E7590841
:105120000139584820F8112055E75A49098841F2B9
:105130001110814216D04DF6DD5081422DD013F072
:10514000010F45D0590801394E4C34F8110000EBDD
:10515000022224F8112001334C4A13804E4B0022C6
:105160001A7078E613F0010F11D05B08013B454837
:1051700030F8131001EB022220F81320424B0122D9
:105180001A700023414A1380414A137063E65B089A
:10519000013B3C4921F81320F0E713F0010F11D037
:1051A0005B08013B374830F8131001EB022220F86E
:1051B0001320354B0F221A700023344A1380344ACF
:1051C000137048E65B08013B2E4921F81320F0E7F5
:1051D000590801392B4820F81120BCE72D490888CF
:1051E00047F27771884212D013F0010F2AD0590884
:1051F0000139244C34F8110000EB022224F811206C
:105200000133224A1380244B00221A7023E613F044
:10521000010F11D05B08013B1A4830F8131001EB65
:10522000022220F81320184B08221A700023174A74
:105230001380174A13700EE65B08013B114921F8F1
:105240001320F0E7590801390E4820F81120D7E75C
:1052500013F0010F0FD0590801390A4C34F811002E
:1052600000EB022224F811200133084A13800A4B74
:1052700000221A70EFE559080139024820F8112080
:10528000F2E700BF9802002008030020DC020020A3
:10529000E1020020DA0200200603002000B583B0FE
:1052A000304BDB6913F0200F07D02E4B1B6813F037
:1052B000200F02D0FFF796FD33E02A4BDB6913F095
:1052C000080F25D1274BDB6913F0020F2CD1254B9A
:1052D000DB6913F0040F31D1224BDB6913F0010FAE
:1052E00036D1214BDB6913F0400F1AD01E4B1B68DF
:1052F00013F0400F15D01B4B40221A62194A52E896
:10530000003F23F0400342E800310029F6D108E0D5
:10531000144B5B6A9DF8072052FA83F3DBB28DF8D9
:10532000073003B05DF804FB0E4B5B6A9DF8072065
:1053300052FA83F3DBB28DF80730F2E7094B5B6A70
:105340009DF8072052FA83F3DBB28DF80730E8E7C7
:10535000044B5B6A9DF8072052FA83F3DBB28DF8A9
:105360000730DEE70010014000140140024B4FF00F
:105370000062DA60704700BF0064024008B50A4B63
:105380005B6813F0006F09D1074B5B6813F0007F77
:1053900003D0054B4FF00072DA6008BDFFF7E6FF5F
:1053A000024B00221A70F8E700640240E00200207D
:1053B00082B00A4B1A6C42F080521A641A6C02F0E6
:1053C00080520092009A5A6C42F480425A645B6C9C
:1053D00003F480430193019B02B070470038024000
:1053E00030B58DB000230793089309930A930B936C
:1053F0000368384A934204D0374A934246D00DB0EE
:1054000030BD364B5A6C42F480725A645A6C02F4C6
:1054100080720192019A1A6B42F004021A631A6BAD
:1054200002F004020292029A1A6B42F001021A631D
:105430001A6B02F001020392039A1A6B42F0020205
:105440001A631B6B03F002030493049B0324079469
:10545000089407A9224801F087FB042307930894C6
:105460000025099507A91F4801F07EFB07940894C1
:10547000099507A91C4801F077FB2A462946122006
:1054800001F00CFD122001F019FDB8E7134B5A6C26
:1054900042F480625A645A6C02F480620592059A62
:1054A0001A6B42F020021A631B6B03F02003069371
:1054B000069B202307930323089307A90B4801F0B9
:1054C00053FB00221146122001F0E8FC122001F0EB
:1054D000F5FC94E700200140002201400038024022
:1054E0000008024000000240000402400014024094
:1054F000F0B5ADB0044600212791289129912A9159
:105500002B91902203A8FBF727F92268224B9A429D
:1055100001D02DB0F0BD4FF42003039303A801F098
:1055200023F8002835D11D4B5A6C42F400625A64AE
:105530005A6C02F400620092009A1A6B42F0040264
:105540001A631A6B02F004020192019A1A6B42F07C
:1055500008021A631B6B03F008030293029B4FF4CB
:10556000F8532793022728970026299603252A9582
:105570000C242B9427A90A4801F0F6FA0423279358
:10558000289729962A952B9427A9064801F0ECFA2A
:10559000BFE7FEF7BDF8C6E7002C01400038024027
:1055A00000080240000C024000B587B00368304A92
:1055B00093421ED02F4A934228D02F4A934230D094
:1055C0002E4A934240D02E4A93421CD12D4B5A6C06
:1055D00042F480225A645B6C03F480230593059B9C
:1055E000002211461A2001F059FC1A2001F066FC35
:1055F00009E0244B1A6C42F004021A641B6C03F09D
:1056000004030193019B07B05DF804FB1D4B5A6C2A
:1056100042F001025A645B6C03F001030293029BA7
:10562000F1E7184B5A6C42F002025A645B6C03F0CB
:1056300002030393039B002211462C2001F02EFC51
:105640002C2001F03BFCDEE70E4B5A6C42F400329A
:105650005A645B6C03F400330493049B00221146EC
:10566000192001F01BFC192001F028FCCBE700BF3A
:1056700000080040000001400004014000440140D7
:10568000004801400038024000B589B00023039370
:1056900004930593069307930368274A934208D01F
:1056A000264A93421AD0264A93422FD009B05DF879
:1056B00004FB244B1A6B42F002021A631B6B03F0CB
:1056C00002030093009B4FF480730393022304931F
:1056D000079303A91C4801F047FAE7E7194B1A6B37
:1056E00042F010021A631B6B03F010030193019B3D
:1056F0004FF40073039302230493032306930123BF
:10570000079303A9114801F02FFACFE70D4B1A6B4D
:1057100042F002021A631B6B03F002030293029B26
:105720004FF400730393022304930323079303A905
:10573000054801F019FAB9E70008004000000140EF
:1057400000480140003802400004024000100240BE
:1057500010B5ACB0044600212791289129912A91D7
:105760002B91902203A8FAF7F7FF2268174B9A4271
:1057700001D02CB010BD4FF40053039303A800F0E8
:10578000F3FE00BB124B1A6C42F000421A641A6C12
:1057900002F000420192019A1A6B42F010021A6361
:1057A0001B6B03F010030293029B03232793022237
:1057B0002892002229922A9308232B9327A905488F
:1057C00001F0D2F9D5E7FDF7A3FFDBE7007C00404D
:1057D00000380240001002404A4B5A6822F440321E
:1057E0005A605A6841680A435A600268536823F451
:1057F0008073536002685368016943EA0123536070
:105800000268536823F040735360026853688168EC
:105810000B4353600268936823F40063936002684B
:105820009368C1680B439360826A374B9A4257D0A2
:105830000268936823F07063936002689368816ADA
:105840000B4393600268936823F0405393600268AF
:105850009368C16A0B4393600268936823F0020364
:10586000936002689368816943EA4103936090F80A
:105870002030002B3FD00268536843F4006353602C
:105880000268536823F46043536001684B68426ABE
:10589000013A43EA42334B600268D36A23F470034F
:1058A000D3620168CB6AC269013A43EA0253CB6210
:1058B0000268936823F4007393600268936890F819
:1058C000301043EA412393600268936823F48063B5
:1058D000936002689368416943EA8123936070474B
:1058E0000268936823F0706393600268936823F002
:1058F00040539360B0E70268536823F40063536039
:10590000CAE700BF002301400100000F28B310B513
:105910000446036C43B1236C13F0100F0BD001202D
:10592000002384F83C3010BDFFF75AFD0023636468
:1059300084F83C30EFE7226C094B134043F002033C
:1059400023642046FFF748FF00206064236C23F0A7
:10595000030343F001032364E2E70120704700BF23
:10596000FDEEFFFF82B00023019390F83C30012B45
:105970007ED0012380F83C3003689A6812F0010F52
:1059800013D19A6842F001029A603D4B1B683D4A70
:10599000A2FB03239B0C03EB4303019302E0019B57
:1059A000013B0193019B002BF9D103689A6812F027
:1059B000010F52D0016C344A0A4042F480720264F2
:1059C0005A6812F4806F05D0026C22F4405242F4FF
:1059D00080520264026C12F4805F19D0426C22F093
:1059E00006024264002280F83C206FF022021A6016
:1059F000264B5B6813F01F0F0DD103689A6812F0F5
:105A0000405F37D19A6842F080429A6000202DE0D2
:105A100000224264E6E703681D4A93420AD01B4B0A
:105A20005B6813F0100F27D103681A4A93420AD01B
:105A300000201BE09A6812F0405FF0D19A6842F0B3
:105A400080429A60EBE79A6812F0405F16D19A683C
:105A500042F080429A60002008E0036C43F010039B
:105A60000364436C43F001034364002002B07047B9
:105A70000220FBE70020F9E70020F7E70020F5E728
:105A80005800002083DE1B43FEF8FFFF0023014087
:105A9000002001400022014090F83C30012B17D03B
:105AA000012380F83C300268936823F0010393607F
:105AB00003689B6813F0010F05D1026C054B13407E
:105AC00043F001030364002380F83C30184670471C
:105AD00002207047FEEEFFFF70B504460D460368D6
:105AE0009A6812F4806F03D09B6813F4807F19D1F9
:105AF00001F044FA064623681A6812F0020F20D11A
:105B0000B5F1FF3FF7D0B5B923681B6813F0020F5A
:105B1000F1D1236C43F004032364002384F83C3068
:105B2000032033E0036C43F020030364002380F878
:105B30003C3001202AE001F021FA801BA842DAD98A
:105B4000E2E76FF012021A60236C43F400732364DF
:105B500023689A6812F0405F17D1A269BAB9DA6A6D
:105B600012F4700F03D09B6813F4806F11D1236C73
:105B700023F480732364236C13F4805F0BD1236CB4
:105B800043F001032364002000E0002070BD0020EA
:105B9000FCE70020FAE70020F8E70368D86C7047BC
:105BA00070477047704770B5044603681E685D68AB
:105BB000C5F3401212EA56022CD0026C12F0100FFC
:105BC00003D1026C42F4007202649A6812F0405FE2
:105BD00019D1A269BAB9DA6A12F4700F03D09A68BF
:105BE00012F4806F0FD15A6822F020025A60236CA1
:105BF00023F480732364236C13F4805F03D1236C3C
:105C000043F0010323642046FFF7CAFF23686FF0C7
:105C100012021A60C5F3C01313EA960335D0236C41
:105C200013F0100F03D1236C43F400532364236853
:105C30009A6812F4401F21D19A6B12F4401F03D0CE
:105C40009A6812F4806F19D15A6812F4806F15D1D6
:105C50009A6812F0405F11D1A2697AB95A6822F0AD
:105C600080025A60236C23F480532364236C13F462
:105C7000807F03D1236C43F001032364204600F0AE
:105C80001FF923686FF00C021A60C5F380131E42DF
:105C900004D023681B6813F0010F05D1C5F380659C
:105CA00015EA56150CD170BD236C43F48033236480
:105CB0002046FFF776FF23686FF001021A60EDE7D8
:105CC000636C43F00203636423686FF020051D607A
:105CD0002046FFF767FF23681D60E4E730B482B019
:105CE0000022019290F83C20012A00F0DC8003465B
:105CF000012280F83C200A68B2F1004F18BF092A3F
:105D000022D90468E06892B202EB42021E3A4FF0D8
:105D1000070C0CFA02F220EA0202E2600A68634809
:105D200082420AD01D68E8688C6892B202EB420297
:105D30001E3A94402043E8601CE01868C2688C68F2
:105D400042EA0462C26015E00468206992B202EB84
:105D500042024FF0070C0CFA02F220EA0202226122
:105D60001C6820690A8802EB42028D6805FA02F27B
:105D7000024322614A68062A29D81C68606B02EB3C
:105D80008202053A4FF01F0C0CFA02F220EA0202DE
:105D900062631C68606B4A6802EB8202053AB1F8E4
:105DA00000C00CFA02F2024362631868404A904253
:105DB0003DD018683E4A904243D018683C4A904211
:105DC0004CD0002083F83C0002B030BC70470C2A55
:105DD00016D81D68286B02EB8202233A1F2404FAAE
:105DE00002F220EA02022A631D68286B4A6802EB6D
:105DF0008202233A0C8804FA02F202432A63D4E7AF
:105E00001D68E86A02EB8202413A1F2404FA02F29A
:105E100020EA0202EA621D68E86A4A6802EB82022E
:105E2000413A0C8804FA02F20243EA62BDE70A68CA
:105E3000B2F1004FBDD11F48426822F440024260D7
:105E4000B7E70A68122AB8D11A4A506820F400004D
:105E50005060506840F480005060AEE70A68134814
:105E6000112A18BF8242ACD1124A506820F4800037
:105E70005060506840F40000506009680B4A91423D
:105E80009FD10D4A12680D49A1FB0212920C02EB40
:105E900082025200019202E0019A013A0192019AB3
:105EA000002AF9D18DE702208EE700BF1200001012
:105EB00000200140002301405800002083DE1B43E6
:105EC00070470000002800F0068270B582B00446DA
:105ED000036813F0010F29D0954B9B6803F00C0366
:105EE000042B1AD0924B9B6803F00C03082B0FD0A5
:105EF0006368B3F5803F40D0002B54D18C4B1A68B7
:105F000022F480321A601A6822F480221A6039E082
:105F1000874B5B6813F4800FEAD0854B1B6813F442
:105F2000003F03D06368002B00F0D781236813F093
:105F3000020F74D07E4B9B6813F00C0F5ED07C4B2D
:105F40009B6803F00C03082B53D0E368002B00F090
:105F50008980774A136843F00103136001F00EF85B
:105F60000546734B1B6813F0020F72D101F006F85F
:105F7000401B0228F5D90320B4E16D4A136843F4AD
:105F80008033136063682BB300F0F8FF0546684B5D
:105F90001B6813F4003FC9D100F0F0FF401B6428D8
:105FA000F5D903209EE1B3F5A02F09D0604B1A6804
:105FB00022F480321A601A6822F480221A60E1E723
:105FC0005B4B1A6842F480221A601A6842F48032ED
:105FD0001A60D7E700F0D2FF0546554B1B6813F453
:105FE000003FA3D000F0CAFF401B6428F5D903206E
:105FF00078E14F4B5B6813F4800FA6D14C4B1B68C4
:1060000013F0020F03D0E368012B40F06881484A87
:10601000136823F0F803216943EAC103136023687E
:1060200013F0080F46D0636983B3414A536F43F0BE
:106030000103536700F0A2FF05463D4B5B6F13F071
:10604000020F37D100F09AFF401B0228F5D9032038
:1060500048E1374A136823F0F803216943EAC10392
:106060001360DCE7324A136823F00103136000F089
:1060700085FF05462E4B1B6813F0020FCFD000F0B2
:106080007DFF401B0228F5D903202BE1284A536FDE
:1060900023F00103536700F071FF0546244B5B6F4B
:1060A00013F0020F06D000F069FF401B0228F5D95B
:1060B000032017E1236813F0040F7DD01C4B1B6CE9
:1060C00013F0805F1ED11A4B1A6C42F080521A6492
:1060D0001B6C03F080530193019B0125154B1B683A
:1060E00013F4807F10D0A368012B25D0002B3BD167
:1060F0000F4B1A6F22F001021A671A6F22F0040286
:106100001A671EE00025E9E70A4A136843F4807322
:10611000136000F033FF0646064B1B6813F4807FC4
:10612000E1D100F02BFF801B6428F5D90320D9E0D2
:106130000038024000700040724A136F43F00103C0
:106140001367A36833B300F019FF06466D4B1B6F4E
:1061500013F0020F2FD100F011FF801B41F28833A2
:106160009842F3D90320BDE0052B09D0654B1A6F87
:1061700022F001021A671A6F22F004021A67E0E7A0
:10618000604B1A6F42F004021A671A6F42F0010264
:106190001A67D6E700F0F2FE06465A4B1B6F13F063
:1061A000020F08D000F0EAFE801B41F288339842CB
:1061B000F3D9032096E0FDB9A369002B00F091808C
:1061C000504A926802F00C02082A59D0022B19D0CA
:1061D0004C4A136823F08073136000F0CFFE04462E
:1061E000484B1B6813F0007F48D000F0C7FE001B2F
:1061F0000228F5D9032075E0424A136C23F080533E
:106200001364D9E73F4A136823F08073136000F0EA
:10621000B5FE05463B4B1B6813F0007F06D000F02F
:10622000ADFE401B0228F5D903205BE0E369226A3A
:106230001343626A43EA8213A26A5208013A43EAAC
:106240000243E26A43EA0263226B43EA02732D4A85
:106250005360136843F08073136000F08FFE0446B0
:10626000284B1B6813F0007F06D100F087FE001B4F
:106270000228F5D9032035E0002033E0002031E08A
:10628000204A5268012B2FD002F48003E1698B422F
:106290002CD102F03F03216A8B4229D1616A47F673
:1062A000C0731340B3EB811F24D102F44031A36AC1
:1062B0005B08013BB1EB034F1ED102F07063E16A52
:1062C000B3EB016F1AD102F0E042236BB2EB037F14
:1062D00016D1002006E001207047012002E00120D5
:1062E00000E0002002B070BD0120FBE70120F9E7CB
:1062F0000120F7E70120F5E70120F3E70120F1E7AE
:106300000120EFE70038024008B5264B9B6803F0F8
:106310000C03042B41D0082B41D1224B5A6802F0C8
:106320003F025B6813F4800F12D01E4B5968C1F313
:1063300088111D480023A1FB0001FAF707FF194B44
:106340005B68C3F3014301335B00B0FBF3F008BDAE
:10635000144B5868C0F388104FEA401CBCEB000C8B
:106360006EEB0E0E4FEA8E1343EA9C634FEA8C11DC
:10637000B1EB0C0163EB0E03DB0043EA5173C90080
:1063800011EB000C43F10003990200234FEA8C202B
:1063900041EA9C51FAF7DAFED1E70348D7E7034810
:1063A000D5E700BF0038024040787D010024F400AA
:1063B000002800F0A08070B50D460446524B1B68C3
:1063C00003F00F038B420BD24F4A136823F00F03E5
:1063D0000B431360136803F00F038B4240F08D8072
:1063E000236813F0020F17D013F0040F04D0474AAC
:1063F000936843F4E0539360236813F0080F04D0CC
:10640000424A936843F460439360404A936823F0A0
:10641000F003A1680B439360236813F0010F31D0A0
:106420006368012B20D0022B25D0384A126812F065
:10643000020F64D035498A6822F0030213438B604F
:1064400000F09CFD0646314B9B6803F00C0362682C
:10645000B3EB820F16D000F091FD801B41F2883320
:106460009842F0D9032045E0284A126812F4003F10
:10647000E0D101203EE0254A126812F0007FD9D118
:10648000012037E0204B1B6803F00F03AB420AD911
:106490001D4A136823F00F032B431360136803F0A6
:1064A0000F03AB422DD1236813F0040F06D0174A17
:1064B000936823F4E053E1680B439360236813F07F
:1064C000080F07D0114A936823F46043216943EA17
:1064D000C1039360FFF718FF0C4B9B68C3F30313D2
:1064E0000B4AD35CD8400B4B18600B4B186800F07C
:1064F00007FD002070BD012070470120FAE7012050
:10650000F8E70120F6E700BF003C024000380240F7
:1065100080C000085800002054000020014B18687B
:10652000704700BF5800002008B5FFF7F7FF044B85
:106530009B68C3F38223034AD35CD84008BD00BFE5
:106540000038024078C0000808B5FFF7E7FF044BA9
:106550009B68C3F34233034AD35CD84008BD00BFF5
:106560000038024078C00008F0B583B004460668E1
:1065700016F001060DD0B54B9A6822F400029A601D
:106580009A68416B0A439A60436B002B00F0678165
:106590000026256815F4002511D0AC4AD2F88C30BD
:1065A00023F44013E16B0B43C2F88C30E36BB3F57B
:1065B000801F00F05681002B00F0558100252368D4
:1065C00013F4801F0FD0A14AD2F88C3023F440037B
:1065D000216C0B43C2F88C30236CB3F5800F00F0B4
:1065E000448103B90125236813F0807F00D0012680
:1065F00013F0200F40F03B81236813F0100F0CD0F4
:10660000924BD3F88C2022F08072C3F88C20D3F800
:106610008C20A16B0A43C3F88C20236813F4804FAD
:1066200008D08A4AD2F8903023F44033616E0B438D
:10663000C2F89030236813F4004F08D0834AD2F890
:10664000903023F44023A16E0B43C2F890302368AE
:1066500013F4803F08D07D4AD2F8903023F44013E1
:10666000E16E0B43C2F89030236813F4003F08D06A
:10667000764AD2F8903023F44003216F0B43C2F8DE
:106680009030236813F0400F08D0704AD2F8903051
:1066900023F00303616C0B43C2F89030236813F0BE
:1066A000800F08D0694AD2F8903023F00C03A16C17
:1066B0000B43C2F89030236813F4807F08D0634AFC
:1066C000D2F8903023F03003E16C0B43C2F89030E5
:1066D000236813F4007F08D05C4AD2F8903023F08E
:1066E000C003216D0B43C2F89030236813F4806F10
:1066F00008D0564AD2F8903023F44073616D0B43B2
:10670000C2F89030236813F4006F08D04F4AD2F8D3
:10671000903023F44063A16D0B43C2F8903023689E
:1067200013F4805F08D0494AD2F8903023F44053E4
:10673000E16D0B43C2F89030236813F4005F08D07A
:10674000424AD2F8903023F44043216E0B43C2F802
:106750009030236813F4800F08D03C4AD2F8903070
:1067600023F08063A16F0B43C2F89030236813F4C9
:10677000001F0DD0354AD2F8903023F00063E16F4E
:106780000B43C2F89030E36FB3F1006F00F0D58097
:10679000236813F0080F00D0012513F4802F08D0D0
:1067A0002A4AD2F8903023F04073616F0B43C2F84D
:1067B0009030236813F4000F09D0244AD2F89030A7
:1067C00023F08053D4F880100B43C2F89030236834
:1067D00013F0806F09D01D4AD2F8903023F0005397
:1067E000D4F884100B43C2F89030236813F0006F84
:1067F00009D0164AD2F88C3023F00073D4F88810F0
:106800000B43C2F88C30236813F0805F09D00F4A25
:10681000D2F88C3023F08063D4F88C100B43C2F88C
:106820008C3026B9236813F0007F00F00681074AF8
:10683000136823F08063136000F0A0FB0646034B4F
:106840001B6813F0006F7AD002E000BF00380240EE
:1068500000F094FB801B6428F1D90320F0E00126AE
:1068600097E60126A7E60125A9E60126B9E67F4BB2
:106870001A6C42F080521A641B6C03F0805301932F
:10688000019B7B4A136843F48073136000F076FB2E
:106890000746774B1B6813F4807F06D100F06EFB30
:1068A000C01B6428F5D90320CAE0704B1B6F13F49A
:1068B000407315D0226B02F440729A4210D06B4B99
:1068C0001A6F22F44072196F41F480311967196F01
:1068D00021F4803119671A671B6F13F0010F12D171
:1068E000236B03F44072B2F5407F1DD05F4A93687A
:1068F00023F4F81393605D490B6F226BC2F30B0214
:1069000013430B6778E600F039FB0746574B1B6FC4
:1069100013F0020FE4D100F031FBC01B41F28833C9
:106920009842F3D903208BE05048826822F4F81291
:10693000504919400A438260DDE7012528E72368B2
:1069400013F0010F13D0636B8BB9484AD2F884302F
:10695000D2F88410606803F4403343EA801301F0F6
:1069600070610B43A16843EA0173C2F88430236865
:1069700013F4002F03D0E26BB2F5801F06D013F49E
:10698000801F1ED0236CB3F5800F1AD1374AD2F87E
:106990008430D2F88410606803F4403343EA8013F3
:1069A000E06843EA006301F0E0410B43C2F8843041
:1069B000D2F88C3023F01F03616A01390B43C2F80F
:1069C0008C30236813F0807F11D0284AD2F88400DD
:1069D000D2F88410666823691B0443EA861300F02A
:1069E0007060034301F0E0410B43C2F88430236838
:1069F00013F0007F0DD0626823691B0443EA821301
:106A0000E26843EA0263A26843EA0273174AC2F8E3
:106A10008430164A136843F08063136000F0AEFAC6
:106A20000646124B1B6813F0006F06D100F0A6FA61
:106A3000801B6428F5D9032002E0012D02D000203C
:106A400003B0F0BD094A136823F08053136000F0CF
:106A500095FA0546054B1B6813F0005F0CD000F05B
:106A60008DFA401B6428F5D90320E9E7003802407D
:106A700000700040FFFCFF0F236813F4002F01D0CB
:106A8000E26B22B113F4801F1DD0236CDBB9354AB1
:106A9000D2F88830D2F88810606903F4403343EAB2
:106AA0008013A06943EA006301F0E0410B43C2F8A0
:106AB0008830D2F88C3023F4F853A16A013943EAC4
:106AC0000123C2F88C30236813F4001F03D0E36F56
:106AD000B3F1006F31D0236813F0080F19D0214AA9
:106AE000D2F88810D2F88830606903F4403343EA62
:106AF000801301F070610B43E16943EA0173C2F84E
:106B00008830D2F88C3023F44033E16A0B43C2F86A
:106B10008C30144A136843F08053136000F02EFA4F
:106B20000446104B1B6813F0005F19D100F026FAE1
:106B3000001B6428F5D9032082E70A4AD2F88800AE
:106B4000D2F888106569236A1B0443EA851300F0B4
:106B50007060034301F0E0410B43C2F88830BAE7AC
:106B600000206DE70038024000230F2B00F2F48074
:106B700070B582B066E085684FEA430E032404FADC
:106B80000EF425EA0405CC6804FA0EF42C43846064
:106B9000446824EA02044A68C2F300129A4022437D
:106BA00042605DE0DC08083450F8242003F007055B
:106BB000AD004FF00F0E0EFA05FE22EA0E0E0A6926
:106BC000AA4042EA0E0240F824205DE0092200E0DB
:106BD000002202FA0EF22A430234604D45F82420C6
:106BE0005F4A94686FEA0C0224EA0C054E6816F4BA
:106BF000801F01D04CEA0405594CA560E46802EA04
:106C000004054E6816F4001F01D04CEA0405544CEC
:106C1000E560646802EA04054E6816F4003F01D09E
:106C20004CEA04054E4C6560246822404D6815F41A
:106C3000803F01D04CEA0402494C226001330F2B03
:106C400000F2888001229A400C6804EA020C32EAC1
:106C50000404F3D14C6804F00304013C012C8AD9EC
:106C60004A6802F00302032A09D0C4685D000322C7
:106C7000AA4024EA02048A68AA402243C2604A6801
:106C800002F00302022A8DD004684FEA430E032269
:106C900002FA0EF224EA02044A6802F0030202FA3F
:106CA0000EF2224302604A6812F4403FC6D02D4AD9
:106CB000546C44F480445464526C02F48042019257
:106CC000019A9C08A51C254A52F8255003F0030E92
:106CD0004FEA8E0E0F2202FA0EF225EA0205224A30
:106CE00090423FF475AF02F58062904222D002F5E7
:106CF0008062904220D002F5806290421ED002F560
:106D0000806290421CD002F5806290421AD002F557
:106D10008062904218D002F58062904216D002F54F
:106D20008062904214D002F5806290423FF44EAFF0
:106D30000A224EE701224CE702224AE7032248E7F3
:106D4000042246E7052244E7062242E7072240E7FD
:106D500008223EE702B070BD704700BF0038014016
:106D6000003C014000380240000002400369194223
:106D700001D001207047002070470AB1816170473F
:106D8000090481617047436901EA030221EA0301B2
:106D900041EA02418161704710B582B01B4B1A6C09
:106DA00042F080521A641B6C03F080530193019BE4
:106DB000174A136843F48033136000F0DFF8044689
:106DC000134B5B6813F4803F08D100F0D7F8001B29
:106DD000B0F57A7FF4D9032002B010BD0C4A1368D5
:106DE00043F40033136000F0C9F80446084B5B68B5
:106DF00013F4003F07D100F0C1F8001BB0F57A7F13
:106E0000F4D90320E8E70020E6E700BF003802409D
:106E100000700040002804DB0901C9B2044B19547A
:106E2000704700F00F000901C9B2024B19547047B6
:106E300000E400E014ED00E000B500F00700C0F150
:106E4000070CBCF1040F28BF4FF0040C031D062BE8
:106E50000FD9C31E4FF0FF3E0EFA0CF021EA0001DD
:106E600099400EFA03FE22EA0E0241EA02005DF8A2
:106E700004FB0023EEE700000649CB6823F4E0633F
:106E80001B041B0C000200F4E0600343024A1A4397
:106E9000CA60704700ED00E00000FA0510B5044636
:106EA000054BD868C0F30220FFF7C6FF0146204615
:106EB000FFF7B0FF10BD00BF00ED00E0002807DBCA
:106EC00000F01F02400901239340024A42F820309B
:106ED000704700BF00E100E00138B0F1807F0BD2C5
:106EE0004FF0E0235861054AF02182F8231000207A
:106EF000986107221A6170470120704700ED00E099
:106F000010B504460E4B1A784FF47A73B3FBF2F3C4
:106F10000C4A1068B0FBF3F0FFF7DEFF68B90F2CE6
:106F200001D901200AE0002221464FF0FF30FFF78F
:106F3000B5FF054B1C60002000E0012010BD00BF24
:106F400051000020580000205400002008B5032004
:106F5000FFF792FF0020FFF7D3FFFEF729FA00208A
:106F600008BD0000034A1168034B1B780B441360F3
:106F7000704700BF5C06002051000020014B1868DC
:106F8000704700BF5C06002038B50446FFF7F6FFE7
:106F90000546B4F1FF3F02D0044B1B781C44FFF7B9
:106FA000EDFF401BA042FAD338BD00BF51000020C6
:106FB000034B9B68C3F30313024AD35CD84070476A
:106FC0000038024080C00008034B9B68C3F3822353
:106FD000024AD35CD84070470038024078C00008AD
:106FE000034B9B68C3F34233024AD35CD8407047DB
:106FF0000038024078C000080D4B5B6803F4800342
:107000009BB90C480A4B5A6802F03F02B0FBF2F001
:107010005A68C2F3881202FB00F05B68C3F30143B5
:1070200001335B00B0FBF3F070470348EAE700BFB1
:10703000003802400024F40040787D0108B5074B79
:107040009B6803F00C03042B04D0082B04D1FFF73A
:10705000D3FF08BD0248FCE70248FAE700380240C7
:1070600040787D010024F40008B5032808D00C28DE
:107070002ED0B0F5406F53D030287AD0002008BD14
:10708000514BD3F89030034043EA00434F4A9342B8
:1070900008D0B3F1031F0CD0013A934211D1FFF78E
:1070A000CDFFECE7484B186810F00200E7D04848E5
:1070B000E5E7454B186F10F00200E0D04FF40040B8
:1070C000DDE7FFF7BBFFFFF773FFFFF789FFD6E7A9
:1070D0003D4BD3F89030034043EA00433D4A93428E
:1070E00008D0B3F10C1F0CD0043A934211D1FFF732
:1070F000A5FFC4E7344B186810F00200BFD0344835
:10710000BDE7314B186F10F00200B8D04FF40040CB
:10711000B5E7FFF793FFFFF74BFFFFF755FFAEE72C
:10712000294BD3F89030034043EA00432A4A934264
:1071300009D0B3F10C2F0DD0A2F58062934211D18A
:10714000FFF77CFF9BE7204B186810F0020096D0F9
:107150001F4894E71C4B186F10F002008FD04FF4BB
:1071600000408CE7FFF76AFFFFF722FFFFF738FFC9
:1071700085E7154BD3F89030034043EA0043174AA4
:10718000934208D0B3F1301F0DD0103A934213D17F
:10719000FFF754FF73E70C4B186810F002003FF440
:1071A0006EAF0B486BE7084B186F10F002003FF40E
:1071B00066AF4FF4004062E7FFF740FFFFF7F8FECD
:1071C000FFF702FF5BE700BF003802400200030048
:1071D0000024F40008000C000008000C200030001F
:1071E00008B5C0280AD0B0F5407F2FD0B0F5405F79
:1071F00055D0B0F5404F7BD0002008BD524BD3F89E
:107200009030034043EA0043504A934208D0B3F120
:10721000C01F0CD0403A934211D1FFF70FFFECE7AB
:10722000494B186810F00200E7D04948E5E7464BA3
:10723000186F10F00200E0D04FF40040DDE7FFF7D8
:10724000FDFEFFF7B5FEFFF7BFFED6E73E4BD3F8D6
:107250009030034043EA00433E4A934209D0B3F1E1
:10726000032F0DD0A2F58072934211D1FFF7E6FEF5
:10727000C3E7354B186810F00200BED03448BCE7B5
:10728000314B186F10F00200B7D04FF40040B4E754
:10729000FFF7D4FEFFF78CFEFFF796FEADE72A4B13
:1072A000D3F89030034043EA00432B4A934209D07D
:1072B000B3F1302F0DD0A2F58052934211D1FFF7D8
:1072C000BDFE9AE7204B186810F0020095D02048C8
:1072D00093E71D4B186F10F002008ED04FF4004062
:1072E0008BE7FFF7ABFEFFF763FEFFF76DFE84E76A
:1072F000154BD3F89030034043EA0043174A9342BA
:1073000009D0B3F1C02F0ED0A2F58042934213D121
:10731000FFF794FE71E70C4B186810F002003FF481
:107320006CAF0B4869E7084B186F10F002003FF490
:1073300064AF4FF4004060E7FFF780FEFFF738FED0
:10734000FFF742FE59E700BF003802408000C0004E
:107350000024F4000002000300200030008000C080
:1073600000B5836891FAA1FCBCFA8CFC4FEA4C0C86
:107370004FF0030E0EFA0CFC23EA0C0391FAA1F174
:10738000B1FA81F149008A40134383605DF804FB40
:1073900000B5C36891FAA1FCBCFA8CFC4FEA4C0C16
:1073A0004FF0030E0EFA0CFC23EA0C0391FAA1F144
:1073B000B1FA81F149008A401343C3605DF804FBD0
:1073C00000B5036A91FAA1FCBCFA8CFC4FEA8C0C64
:1073D0004FF00F0E0EFA0CFC23EA0C0391FAA1F108
:1073E000B1FA81F189008A40134303625DF804FB1E
:1073F00000B5436A090A91FAA1FCBCFA8CFC4FEA79
:107400008C0C4FF00F0E0EFA0CFC23EA0C0391FAD1
:10741000A1F1B1FA81F189008A40134343625DF81A
:1074200004FB00B5036891FAA1FCBCFA8CFC4FEA9E
:107430004C0C4FF0030E0EFA0CFC23EA0C0391FAED
:10744000A1F1B1FA81F149008A40134303605DF86C
:1074500004FBF8B507460E460D6895FAA5F5B5FA92
:1074600085F519E0B26821463846FFF779FF3268A2
:10747000F1687B6823EA020301FB02F213437B609D
:1074800016E0726921463846FFF7B2FF726821465E
:107490003846FFF7C6FF0135346834FA05F21BD0D1
:1074A0000122AA401440F6D07368013B012BD9D9C0
:1074B000326921463846FFF76BFF7368022BE5D12E
:1074C00094FAA4F3B3FA83F3072BDAD8726921464E
:1074D0003846FFF775FFD9E70020F8BD0B4B1B6856
:1074E0000B4AA2FB03235B0A41F2883202FB03F33F
:1074F0001A46013B3AB1426B12F0800FF8D0C52317
:107500008363002070474FF0004070475800002010
:10751000D34D621084B00DF1040C8CE80E000B46C4
:107520001343039A1343049A1343059A1343069A89
:1075300013434168034A0A4013434360002004B0E8
:10754000704700BF0081FFFFD0F8800070470B68D4
:10755000C0F880300020704703230360002070478C
:10756000006800F0030070470B6883604B688A680E
:107570001343CA6813430A691343C2686FF30B02CB
:107580001343C360002070470069C0B270471430D5
:10759000405870470B6843624B6883628B68CA68C7
:1075A00013430A6913434A691343C26A22F0F7027C
:1075B0001343C3620020704710B586B00446002311
:1075C00001930293039304934FF48063059301A9FD
:1075D000FFF7CAFF2046FFF781FF06B010BD00008D
:1075E00038B504460D46504B1B685049A1FB0313A8
:1075F0005B0A03FB02F21346013A002B5DD0636B7A
:1076000013F0450FF7D013F4006FF4D1636B13F050
:10761000040F06D1636B13F0010F05D00120A063A6
:107620004DE00420A0634AE0C523A3632046FFF792
:10763000ABFFA84201D0012041E000212046FFF726
:10764000A6FF03463A481840C8B3002B38DB13F0B6
:10765000804F38D113F0005F37D113F0805F36D1FF
:1076600013F0006F36D113F0806F36D113F0807FA6
:1076700036D113F4000F36D113F4800F36D113F442
:10768000001F36D113F4801F36D113F4802F36D16A
:1076900013F4003F36D113F4803F36D113F4004F7A
:1076A00036D113F4804F36D113F4005F36D113F086
:1076B000080F36D04FF4000001E04FF0004038BD15
:1076C0004FF00070FBE74020F9E78020F7E74FF428
:1076D0008070F4E74FF40070F1E74FF48060EEE75C
:1076E0004FF40060EBE74FF48050E8E74FF40050B0
:1076F000E5E74FF48040E2E74FF40040DFE74FF466
:107700000030DCE74FF48020D9E74FF40020D6E7C3
:107710004FF48010D3E74FF40010D0E74FF480000F
:10772000CDE74FF48030CAE758000020D34D6210F7
:1077300008E0FFFD30B587B00446019110250295A1
:1077400040230393002304934FF48063059301A91E
:10775000FFF70AFF41F2883229462046FFF740FF33
:1077600007B030BD30B587B00446019111250295B0
:1077700040230393002304934FF48063059301A9EE
:10778000FFF7F2FE41F2883229462046FFF728FF34
:1077900007B030BD30B587B004460191122502957F
:1077A00040230393002304934FF48063059301A9BE
:1077B000FFF7DAFE41F2883229462046FFF710FF34
:1077C00007B030BD30B587B0044601911825029549
:1077D00040230393002304934FF48063059301A98E
:1077E000FFF7C2FE41F2883229462046FFF7F8FE35
:1077F00007B030BD30B587B0044601911925029518
:1078000040230393002304934FF48063059301A95D
:10781000FFF7AAFE41F2883229462046FFF7E0FE34
:1078200007B030BD30B587B00446002301930C2566
:1078300002954022039204934FF48063059301A9BB
:10784000FFF792FE034A29462046FFF7C9FE07B01C
:1078500030BD00BF00E1F50530B587B004460192A8
:107860000725029540230393002304934FF480637C
:10787000059301A9FFF778FE41F288322946204698
:10788000FFF7AEFE07B030BD30B587B004460191BA
:107890003725029540230393002304934FF480631C
:1078A000059301A9FFF760FE41F288322946204680
:1078B000FFF796FE07B030BD30B587B004460191A2
:1078C0000625029540230393002304934FF480631D
:1078D000059301A9FFF748FE41F288322946204668
:1078E000FFF77EFE07B030BD30B587B004460023F9
:1078F0000193332502954022039204934FF4806351
:10790000059301A9FFF730FE41F28832294620464F
:10791000FFF766FE07B030BD30B587B00446019171
:107920000D25029540230393002304934FF48063B5
:10793000059301A9FFF718FE41F288322946204637
:10794000FFF74EFE07B030BD0146144B1B68144ACA
:10795000A2FB03235B0A41F2883202FB03F31A46BF
:10796000013BBAB14A6B12F0450FF8D012F4006F28
:10797000F5D14B6B13F0040F06D1486B10F00100EA
:1079800005D1C5238B6370470420886370470120AD
:10799000886370474FF00040704700BF58000020D8
:1079A000D34D621010B586B0044600230193022225
:1079B0000292C022039204934FF48063059301A9BD
:1079C000FFF7D2FD2046FFF7BFFF06B010BD10B590
:1079D00086B00446019109230293C0230393002338
:1079E00004934FF48063059301A9FFF7BDFD204682
:1079F000FFF7AAFF06B010BD0146104B1B68104AE6
:107A0000A2FB03235B0A41F2883202FB03F31A460E
:107A1000013B82B14A6B12F0450FF8D012F4006FAF
:107A2000F5D1486B10F0040002D1C5238B63704779
:107A30000420886370474FF00040704758000020D2
:107A4000D34D621010B586B004460A4B0B43019328
:107A50002923029340230393002304934FF480636C
:107A6000059301A9FFF780FD2046FFF7C5FF06B08B
:107A700010BD00BF00001080F8B505460E46174641
:107A8000234B1B68234AA2FB03235B0A41F2883283
:107A900002FB03F31A46013B8AB36C6B14F0450FEB
:107AA000F8D014F4006FF5D16B6B13F0040F06D10E
:107AB0006B6B13F0010F05D00120A86321E00420B7
:107AC000A8631EE02846FFF75FFDB04201D0012009
:107AD00017E0C523AB6300212846FFF758FD034696
:107AE00010F4604008D013F4804F0BD113F4004F12
:107AF0000BD04FF4805004E01B0C3B8001E04FF0B2
:107B00000040F8BD4FF40050FBE74FF48030F8E739
:107B100058000020D34D621070B586B004460D4663
:107B200000230193032602964022039204934FF40C
:107B30008063059301A9FFF717FD2A4631462046C9
:107B4000FFF79AFF06B070BD0146164B1B68164A38
:107B5000A2FB03235B0A41F2883202FB03F31A46BD
:107B6000013BE2B14A6B12F0450FF8D012F4006FFE
:107B7000F5D14B6B13F0040F0BD14B6B13F00103DA
:107B80000AD1486B10F040000BD040228A6318469F
:107B900070470420886370470120886370474FF066
:107BA0000040704758000020D34D621010B586B0D9
:107BB00004464FF4D57301930823029340230393A3
:107BC000002304934FF48063059301A9FFF7CCFCD5
:107BD0002046FFF7B9FF06B010BD000070B582B0B7
:107BE0000446002301930068FFF7E6FC054610B148
:107BF000284602B070BD2068FFF7D8FF38B90123CE
:107C0000A364A36C012B0BD02E46284614E000235E
:107C1000A3642068FFF7D0FC0028F2D00546E7E710
:107C200000212068FFF730FE0028EDD04FF080558E
:107C3000DEE7019B01330193019A4FF6FE739A42EE
:107C400013D896B900212068FFF71EFEE0B912494B
:107C50002068FFF7F7FE0646C0B900212068FFF74D
:107C600096FCC30FE5D01E46E3E7019A4FF6FE737C
:107C70009A420ED810F0804302D001236364B7E724
:107C8000002262641D46B3E70546B1E74FF0805518
:107C9000AEE74FF08075ABE7000010C1F0B589B0DA
:107CA00004460F46FFF76AF9064600230093019346
:107CB00008212068FFF73EFD054610B1284609B0AF
:107CC000F0BD216D09042068FFF7DEFD05460028A0
:107CD000F4D14FF0FF33029308230393302304932E
:107CE00002230593002306930123079302A920682A
:107CF000FFF750FC2068FFF7F7FD054658B1DDE7B8
:107D0000FFF722FC4DF825000135FFF737F9831BFB
:107D1000B3F1FF3F3FD02068436B13F02A0F07D128
:107D2000436B13F4001FEBD1436B13F4005FECD1F2
:107D3000436B13F0080F25D1436B13F0020F24D1CE
:107D4000456B15F0200523D140F23A538363019A25
:107D5000130203F47F0343EA0263110A01F47F4133
:107D60000B4343EA12633B60009A130203F47F0360
:107D700043EA0263110A01F47F410B4343EA1263B1
:107D80007B609BE70825856398E70225856395E777
:107D90002025856392E74FF000458FE710B582B04C
:107DA00004460021009101910068FFF7F0FB10F0FC
:107DB000007F13D169462046FFF770FF80B9019B11
:107DC00013F4802F0ED0216D09042068FFF75CFDAD
:107DD00030B902212068FFF76FFD01E04FF4006029
:107DE00002B010BD4FF08060FAE710B582B00446D3
:107DF0000021009101910068FFF7C9FB10F0007F9E
:107E000013D169462046FFF749FF80B9019B13F45F
:107E1000803F0ED0216D09042068FFF735FD30B991
:107E200000212068FFF748FD01E04FF4006002B038
:107E300010BD4FF08060FAE770B581B104460E4680
:107E4000016D09040068FFF767FD054608B1284683
:107E500070BD00212068FFF79AFB3060F7E74FF014
:107E60000065F4E72DE9F04F87B005460C4616464D
:107E70009B46DDF840A0FFF781F8002C36D0814604
:107E800095F83470FFB2012F40F004810023AB63FA
:107E900006EB0B03EA6D93422ED8032385F83430AA
:107EA0002B680022DA626B6C012B00D076024FF057
:107EB000FF3300934FEA4B23019390230293022355
:107EC0000393002304930123059369462868FFF771
:107ED00061FBBBF1010F14D902232B6331462868E3
:107EE000FFF758FCA0B9DDF8048038E0AB6B43F035
:107EF0000063AB630127D2E0AB6B43F00073AB636D
:107F0000CDE001232B6331462868FFF72BFCE9E71E
:107F10002B68654A9A63AB6B0343AB63012385F817
:107F2000343000232B63BAE02868FFF70DFB207084
:107F3000C0F307236370C0F30743A370000EE07023
:107F40000434A8F104080136072EEDD9FFF716F81E
:107F5000A0EB090050450FD2BAF1000F0CD02868F1
:107F6000466B16F4957615D1436B13F4004FEDD0A4
:107F7000B8F1000FEAD0E7E72B684B4A9A63AB6B86
:107F800043F00043AB63012385F8343000232B63B7
:107F9000032784E0436B13F4807F05D0BBF1010F0E
:107FA00002D96B6C032B38D12B685A6B12F0080F77
:107FB00044D15A6B12F0020F4CD15A6B12F0200FC1
:107FC00054D12868436B13F4001F5BD0B8F1000F45
:107FD00058D0FFF7B9FA2070C0F307236370C0F3DD
:107FE0000743A370000EE0700434A8F10408FEF704
:107FF000C5FFA0EB0900504502D2BAF1000FE0D155
:108000002B68294A9A63AB6B43F00043AB630123AF
:1080100085F8343000232B6341E0FFF703FC03466F
:108020000028C1D02A6820499163AA6B1343AB632F
:10803000012385F8343000232B6330E01A4A9A6319
:10804000AB6B43F00803AB63012385F834300023A6
:108050002B6324E0144A9A63AB6B43F00203AB63D7
:10806000012385F8343000232B6318E00E4A9A630D
:10807000AB6B43F02003AB63012385F8343000235E
:108080002B630CE040F23A538363012385F83430CC
:10809000002704E0AB6B43F00053AB630127384685
:1080A00007B0BDE8F08F00BFFF0540002DE9F04F9D
:1080B0008BB005460C4616469B46DDF850A0FEF7F1
:1080C0005DFF002C37D0804695F83470FFB2012F49
:1080D00040F0E1800023AB6306EB0B03EA6D9342B3
:1080E0002FD8032385F834302B680022DA626B6CBA
:1080F000012B00D076024FF0FF3304934FEA4B235D
:108100000593902306930023079308930123099373
:1081100004A92868FFF73EFABBF1010F16D9202306
:108120002B6331462868FFF765FB0190019BABB9D3
:10813000DDF8149040E0AB6B43F00063AB630127C4
:10814000AEE0AB6B43F00073AB63A9E010232B638D
:1081500031462868FFF736FB0190E7E72B68524A63
:108160009A63AB6B019A1343AB63012385F83430F8
:1081700000232B6394E023780393627843EA02237D
:108180000393A27843EA02430393E27843EA02634B
:1081900003930434A9F1040903A92868FFF7D7F968
:1081A0000136072EE7D9FEF7E9FEA0EB080050459F
:1081B0000FD2BAF1000F0CD02868466B16F48D76FA
:1081C00015D1436B13F4804FEDD0B9F1000FEAD015
:1081D000E7E72B68344A9A63AB6B019A1343AB63AE
:1081E000012385F8343000232B63032758E0436BC9
:1081F00013F4807F05D0BBF1010F02D96B6C032B08
:1082000018D12B685A6B12F0080F24D15A6B12F058
:10821000020F2CD15A6B12F0100F34D0224A9A63FD
:10822000AB6B43F01003AB63012385F834300023BC
:108230002B6335E0FFF7F6FA03460028E1D02A6801
:1082400019499163AA6B1343AB63012385F834305A
:1082500000232B6324E0144A9A63AB6B43F00803BA
:10826000AB63012385F8343000232B6318E00E4AFA
:108270009A63AB6B43F00203AB63012385F83430A0
:1082800000232B630CE040F23A529A63012385F8F5
:108290003430002704E0AB6B43F00053AB6301279D
:1082A00038460BB0BDE8F08FFF0540000346426E34
:1082B000920F0A70426EC2F383624A7090F8672090
:1082C00002F003028A7090F86620CA7090F8652068
:1082D0000A7190F864204A71826E120DCA80B0F85B
:1082E0006A2002F00F020A72826EC2F3C0324A7232
:1082F000826EC2F380328A72826EC2F34032CA72D8
:10830000826EC2F300320A7300224A73426C002A62
:1083100040F08680806E40F6FC7202EA8002D86EE1
:1083200042EA90720A61DA6EC2F3C2620A7593F889
:108330006F2002F007024A75DA6EC2F342528A7564
:10834000DA6EC2F38242CA75DA6EC2F3C2320A76BC
:108350000A6901325A65087E00F007000230824047
:108360005A6591F808C00CF00F0C012000FA0CF0CF
:108370009865400A00FB02F2DA654FF400721A6653
:10838000DA6EC2F380324A76DA6EC2F3C6128A76A9
:10839000DA6E02F07F02CA761A6FD20F0A771A6F6E
:1083A000C2F341724A771A6FC2F382628A771A6FF8
:1083B000C2F38352CA771A6FC2F3405281F8202069
:1083C000002081F82100B3F8722002F0010281F848
:1083D00022201A6FC2F3C03281F823201A6FC2F331
:1083E000803281F824201A6FC2F3403281F82520B0
:1083F0001A6FC2F3003281F826201A6FC2F381226D
:1084000081F827201A6FC2F3012281F828201B6F00
:10841000C3F3460381F82930012381F82A307047DD
:10842000012A11D1826E120402F47C12B0F86E009F
:1084300002430A610A69013292025A65DA654FF411
:1084400000729A651A669BE7026805499163826B20
:1084500042F080528263012083F83400704700BFED
:10846000FF05400070B590B004460123ADF812300E
:108470000068FFF775F800286CD0636C032B45D1BA
:10848000636C032B5DD1636C032B1DD0BDF8121000
:10849000216509042068FFF79AFA054600285BD198
:1084A00000212068FFF773F8606604212068FFF759
:1084B0006EF8A06608212068FFF769F8E0660C21D5
:1084C0002068FFF764F8206704212068FFF75FF851
:1084D000000DE06405A92046FFF7E8FE00283ED124
:1084E000226D120400232068FFF7B6F9054698BBF9
:1084F000234653F8106B93E807008DE80700043417
:1085000094E80E003046FFF705F825E02068FFF7F5
:1085100049FA054600BB00212068FFF738F860677C
:1085200004212068FFF733F8A06708212068FFF7CF
:108530002EF8E0670C212068FFF729F8C4F88000C6
:108540009EE70DF112012068FFF7E6FA05460028C4
:1085500099D001E04FF08065284610B070BD4FF013
:108560008055F9E730B58BB004460023049305939A
:10857000069307930893762309930AAB13E9070040
:108580008DE8070004AB0ECB2068FEF7C3FF18B1DF
:10859000012528460BB030BD05462268536823F4F8
:1085A000807353602068FEF7D7FF2268536843F456
:1085B000807353600220FEF7E7FC2046FFF70EFBB6
:1085C00030B1012584F83450A36B0343A363E0E783
:1085D0002046FFF747FF30B1012584F83450A36BE4
:1085E0000343A363D5E74FF400712068FFF7A2F8B7
:1085F0000028CED0236804499963A36B0343A36387
:10860000012584F83450C4E7FF054000A8B110B537
:10861000044690F8343063B1032384F834302046A4
:10862000FFF7A0FF58B9A0632063012384F834301A
:1086300010BD0377FCF75CFFEEE7012070470120D7
:10864000F6E7436C0B60836C4B60C36C8B60036D0F
:10865000CB60436D0B61836D4B61C36D8B61036EAA
:10866000CB6100207047000030B58BB004460D464A
:10867000032380F83430436C032B1CD0B1F5805FAA
:1086800008D0B1F5006F0AD079B1836B43F0006375
:10869000836314E0836B43F0805383630FE0FFF741
:1086A0007DFBA36B0343A36309E0FFF79EFBA36B72
:1086B0000343A36303E0836B43F080538363A36BA3
:1086C000C3B12368174A9A63012584F834504FF4E4
:1086D00000712068FFF72EF830B1236811499963C3
:1086E000A36B0343A3630125012384F83430284698
:1086F0000BB030BD63680493A3680593E3680693E9
:10870000079563690893A36909930AAB13E9070006
:108710008DE8070004AB0ECB2068FEF7FBFE0025BA
:10872000D5E700BFFF05400010B582B00446002326
:10873000019301A9FFF780FB10B1A36B0343A3636F
:108740000198C0F3432002B010BD00000346026848
:1087500012F0400F36D110B402681D4810400A686C
:108760004C682243CC6822430C6922434C69224363
:108770008C692243CC6922430C6A2243104318605F
:108780005868144A02408868B1F816C040EA0C00E4
:1087900002435A608A68B2F5006F03D25A6842F405
:1087A00080525A600A6AB2F5005F07D00020DA6989
:1087B00022F40062DA615DF8044B70478A8C1A611A
:1087C0000020F4E70120DA6922F40062DA617047E0
:1087D0004000FFFFFBF0FFFF70B4046A036A23F060
:1087E0000103036242688569124B2B400D681D43EB
:1087F00024F002048B6823430F4C104EB04218BF84
:10880000A0420CBF0124002405D123F00803CE6848
:108810001E4326F004032CB122F440724C69144329
:108820008A692243426085614A684263036270BC80
:10883000704700BF8CFFFEFF0000014000040140B4
:1088400070B4036A026A22F4807202624268C569E7
:10885000144C2C400E68264323F400738C6843EAC2
:108860000423114C114DA84218BFA0420CBF012493
:10887000002406D123F40063CD6843EA052323F4E2
:1088800080633CB122F440524C6942EA04128C6984
:1088900042EA04124260C6614A68C263036270BC65
:1088A000704700BF8CFFFEFF000001400004014044
:1088B00070B4036A026A22F4805202624468C56995
:1088C0000D4A2A400D6842EA052223F400538D68C0
:1088D00043EA0533094E0A4DA84218BFB04204D1FD
:1088E00024F480444D6944EA85144460C2614A68B6
:1088F0000264036270BC7047FF8CFFFE0000014001
:108900000004014070B4036A026A22F480320262F9
:108910004468426D0D4D15400A682A4323F4003324
:108920008D6843EA05430A4E0A4DA84218BFB0427B
:1089300004D124F480344D6944EA0524446042653E
:108940004A688265036270BC704700BF8FFFFEFFFC
:10895000000001400004014070B4036A026A22F47E
:10896000801202624468456D0D4A2A400D6842EA51
:10897000052223F400138D6843EA0553094E0A4D7E
:10898000A84218BFB04204D124F480244D6944EABF
:108990008524446042654A68C265036270BC7047C2
:1089A000FF8FFFFE000001400004014010B4036A85
:1089B000046A24F001040462846924F0F00C4CEA97
:1089C000021223F00A030B43826103625DF8044B39
:1089D000704710B4036A046A24F0100404628469C6
:1089E00024F4704C4CEA023223F0A00343EA011352
:1089F000826103625DF8044B7047836823F0700363
:108A00000B4343F00703836070470368196A41F220
:108A10001112114208D1196A40F24442114203D1A5
:108A20001A6822F001021A60012380F83D3000200C
:108A30007047000090F83D30DBB2012B3AD10223A1
:108A400080F83D300268D36843F00103D3600368C7
:108A50001A4AB3F1804F18BF93421DD0A2F57C4251
:108A6000934219D002F58062934215D002F58062DC
:108A7000934211D002F5784293420DD002F5705224
:108A8000934209D0A2F59432934205D01A6842F07D
:108A900001021A60002070479968094A0A40062AB4
:108AA00018BFB2F5803F07D01A6842F001021A6081
:108AB00000207047012070470020704700000140EF
:108AC000070001000268D36823F00103D360036844
:108AD000196A41F21112114208D1196A40F2444256
:108AE000114203D11A6822F001021A60012380F8B2
:108AF0003D3000207047704770477047704770479F
:108B0000704770B504460368DE681D6915F0020FF2
:108B100010D016F0020F0DD06FF002021A6101237F
:108B2000037703689B6913F0030F64D0FFF7E6FF38
:108B30000023237715F0040F12D016F0040F0FD086
:108B400023686FF004021A610223237723689B696C
:108B500013F4407F55D02046FFF7D0FF0023237742
:108B600015F0080F12D016F0080F0FD023686FF021
:108B700008021A61042323772368DB6913F0030FCB
:108B800046D02046FFF7BAFF0023237715F0100FD9
:108B900012D016F0100F0FD023686FF010021A6178
:108BA000082323772368DB6913F4407F37D02046FE
:108BB000FFF7A4FF0023237715F0010F02D016F072
:108BC000010F33D115F4025F02D016F0800F35D1BA
:108BD00015F4807F02D016F0800F37D115F0400FCA
:108BE00002D016F0400F39D115F0200F02D016F048
:108BF000200F3BD170BDFFF780FF2046FFF77FFFBE
:108C000096E72046FFF779FF2046FFF778FFA5E7B4
:108C10002046FFF772FF2046FFF771FFB4E72046BA
:108C2000FFF76BFF2046FFF76AFFC3E723686FF08B
:108C300001021A612046FFF75FFFC3E723686FF464
:108C400002521A61204600F016FCC1E723686FF457
:108C500080721A61204600F00FFCBFE723686FF0B6
:108C600040021A612046FFF74BFFBDE723686FF013
:108C700020021A61204600F0FDFBBBE730B5036817
:108C80003F4A904214BF4FF0000E4FF0010EB0F17A
:108C9000804F14BF72464EF00102AAB9394CA0426F
:108CA00014BF00240124384DA8420DD064B904F14A
:108CB000804404F58234A04214BF0024012405F549
:108CC0000065A84200D01CB123F070034C68234318
:108CD000002A33D12B4A904214BF002201222A4C91
:108CE000A0422BD052BB02F1804202F58232904268
:108CF00014BF0022012204F50064A0421ED0EAB98C
:108D0000224A904214BF0022012204F59A34A04264
:108D100014D09AB91E4A904214BF0022012204F5D1
:108D20000064A0420AD04AB91A4A904214BF0022F5
:108D30000122A4F59634A04200D022B123F4407C55
:108D4000CB6843EA0C0323F080034A6913430360B2
:108D50008A68C2620A6882620F4A904214BF7346F0
:108D60004EF001030BB10B690363012343610369F7
:108D700013F0010F03D0036923F00103036130BD39
:108D80000000014000080040000400400044014091
:108D900000180040002000400004014060B310B5FE
:108DA000044690F83D3013B3022384F83D30214649
:108DB00051F8040BFFF762FF012384F8483084F870
:108DC0003E3084F83F3084F8403084F8413084F8F5
:108DD000423084F8433084F8443084F8453084F8D5
:108DE000463084F8473084F83D30002010BD80F8CC
:108DF0003C30FCF7D9FBD7E70120704760B310B5D2
:108E0000044690F83D3013B3022384F83D302146E8
:108E100051F8040BFFF732FF012384F8483084F83F
:108E20003E3084F83F3084F8403084F8413084F894
:108E3000423084F8433084F8443084F8453084F874
:108E4000463084F8473084F83D30002010BD80F86B
:108E50003C30FFF750FED7E70120704770B4036A3B
:108E6000026A22F01002026242688569144C2C40AA
:108E70000D6844EA052523F020038C6843EA0413B7
:108E8000104C114EB04218BFA0420CBF0124002468
:108E900006D123F08003CE6843EA061323F0400393
:108EA0003CB122F440624C6942EA84028C6942EA95
:108EB0008402426085614A688263036270BC7047C5
:108EC000FF8CFFFE000001400004014038B590F81F
:108ED0003C30012B00F0958004460D46012380F8BC
:108EE0003C30142A00F28880DFE802F00B86868688
:108EF0001F86868634868686488686865D86868632
:108F000071000068FFF768FC2268936943F008036A
:108F100093612268936923F0040393612268936943
:108F200029690B439361002067E00068FFF796FF13
:108F30002268936943F4006393612268936923F480
:108F40008063936122689369296943EA01239361ED
:108F5000002052E00068FFF773FC2268D36943F0F9
:108F60000803D3612268D36923F00403D361226824
:108F7000D36929690B43D36100203EE00068FFF705
:108F800097FC2268D36943F40063D3612268D369F4
:108F900023F48063D3612268D369296943EA0123FA
:108FA000D361002029E00068FFF7ACFC2268536D14
:108FB00043F0080353652268536D23F0040353659F
:108FC0002268536D29690B435365002015E0006842
:108FD000FFF7C2FC2268536D43F4006353652268B7
:108FE000536D23F4806353652268536D296943EA06
:108FF00001235365002000E00120002384F83C3069
:1090000038BD0220FCE710B4846824F47F4C42EAA7
:1090100003220A4342EA0C0282605DF8044B704767
:1090200090F83C30012B76D010B50446012380F82F
:109030003C30022380F83D3002689068374B034093
:1090400093600B68602B4CD023D8402B54D011D8A0
:10905000202B03D00AD80BB1102B05D1194620685C
:10906000FFF7CBFC002028E0012026E0302BF5D0D4
:10907000012022E0502B0AD1CA6849682068FFF716
:1090800095FC50212068FFF7B8FC002015E0012076
:1090900013E0B3F5805F3AD0B3F5005F14D0702BC6
:1090A00037D1CB684A6889682068FFF7ACFF22682F
:1090B000936843F0770393600020012384F83D30E8
:1090C000002384F83C3010BDCB684A68896820686A
:1090D000FFF799FF2268936843F480439360002070
:1090E000EBE7CA6849682068FFF773FC60212068D5
:1090F000FFF783FC0020E0E7CA6849682068FFF7B3
:1091000055FC40212068FFF778FC0020D5E70020BF
:10911000D3E70120D1E70220704700BF8800FEFF9F
:1091200001F01F014FF0010C0CFA01FC036A23EA65
:109130000C030362036A8A40134303627047000012
:1091400010B5044610293CD8DFE801F0093B3B3B51
:109150001F3B3B3B263B3B3B2D3B3B3B340090F8CE
:109160003E30DBB2013B18BF0123002B40F0898069
:10917000102974D8DFE801F02C7373736373737371
:10918000677373736B7373736F0090F83F30DBB268
:10919000013B18BF0123E8E790F84030DBB2013B08
:1091A00018BF0123E1E790F84130DBB2013B18BF63
:1091B0000123DAE790F84230DBB2013B18BF01230C
:1091C000D3E790F84330DBB2013B18BF0123CCE773
:1091D000022384F83E3001222068FFF7A1FF2368B4
:1091E0002A492B4A934218BF8B4203D15A6C42F44E
:1091F00000425A642368254AB3F1804F18BF934256
:1092000031D0A2F57C4293422DD002F58062934288
:1092100029D002F58062934225D002F5784293422C
:1092200021D002F5705293421DD0A2F594329342A0
:1092300019D01A6842F001021A60002022E00223CD
:1092400084F83F30C7E7022384F84030C3E70223A5
:1092500084F84130BFE7022384F84230BBE70223A1
:1092600084F84330B7E799680A4A0A40062A18BFCB
:10927000B2F5803F07D01A6842F001021A60002060
:1092800000E0012010BD0020FCE700BF000001400D
:10929000000401400700010038B504460D460022D5
:1092A0000068FFF73DFF23682449254A934218BF11
:1092B0008B420DD1196A41F21112114208D1196A7B
:1092C00040F24442114203D15A6C22F400425A64E3
:1092D0002368196A41F21112114208D1196A40F249
:1092E0004442114203D11A6822F001021A60102D83
:1092F0001FD8DFE805F0091E1E1E0E1E1E1E121EC0
:109300001E1E161E1E1E1A00012384F83E30002069
:1093100038BD012384F83F30F9E7012384F8403059
:10932000F5E7012384F84130F1E7012384F8423066
:10933000EDE7012384F84330E9E700BF0000014076
:109340000004014090F83C20012A45D070B4034647
:10935000012280F83C20022280F83D2002685068FB
:1093600094681E4E1E4DAA4218BFB24203D120F48B
:1093700070004D68284320F070000D68284350604D
:109380001A681648B2F1804F18BF824217D0A0F574
:109390007C40824213D000F5806082420FD000F5FD
:1093A000806082420BD000F57840824207D000F501
:1093B0007050824203D0A0F59430824204D124F050
:1093C0008004896821439160012283F83D200020B8
:1093D00083F83C0070BC70470220704700000140D9
:1093E0000004014090F83C30012B3CD030B40246E0
:1093F000012380F83C30CB6823F440738868034332
:1094000023F480634868034323F40063086803433C
:1094100023F480530869034323F40053486903434A
:1094200023F48043886A034323F47023886943EA62
:10943000004310680D4D0E4CA04218BFA8420CD13D
:1094400023F470034C6A43EA045323F08073CC691D
:10945000234323F00073096A0B434364002082F81E
:109460003C0030BC70470220704700BF0000014044
:1094700000040140704770477047000030B5036832
:109480003B4A904214BF4FF0000E4FF0010EB0F176
:10949000804F14BF72464EF00102AAB9354CA0426B
:1094A00014BF00240124344DA8420DD064B904F146
:1094B000804404F58234A04214BF0024012405F541
:1094C0000065A84200D01CB123F070034C68234310
:1094D000002A33D1274A904214BF00220122264C91
:1094E000A0422BD052BB02F1804202F58232904260
:1094F00014BF0022012204F50064A0421ED0EAB984
:109500001E4A904214BF0022012204F59A34A04260
:1095100014D09AB91A4A904214BF0022012204F5CD
:109520000064A0420AD04AB9164A904214BF0022F1
:109530000122A4F59634A04200D022B123F4407C4D
:10954000CB684CEA030303608A68C2620A888262BD
:109550000D4A904214BF73464EF001030BB10B69E4
:109560000363436943F001034361002030BD00BF42
:109570000000014000080040000400400044014099
:10958000001800400020004000040140B2F5004FE8
:1095900006D001EB5301B1FBF3F189B2C160704712
:1095A0005A0802EB4102B2FBF3F34FF6F0721A4095
:1095B000C3F342031343C3607047000038B5036828
:1095C00013F0010F62D104460D460368314A1A4078
:1095D0004B68C9680B4329690B43A9690B431A43BC
:1095E0000260AB68426822F44052134343606B69E7
:1095F000826822F4407213438360274B984216D04E
:10960000264B98421BD0264B98421CD0254B9842A3
:109610001DD0254B98421ED0244B984220D0244B7D
:10962000984222D0234B984224D001202FE00320DF
:10963000FDF71AFD60B32B680BBB012027E00C205F
:10964000FDF712FDF6E73020FDF70EFDF2E7C02032
:10965000FDF7C6FDEEE74FF44070FDF7C1FDE9E709
:109660004FF44060FDF700FDE4E74FF44050FDF794
:10967000B7FDDFE74FF44040FDF7B2FDDAE7AA6936
:1096800001462046FFF782FF002000E0012038BDA0
:109690000120FCE7F369FFEF0010014000440040A7
:1096A00000480040004C00400050004000140140C1
:1096B00000780040007C0040034AD2F8883043F430
:1096C0007003C2F88830704700ED00E008B501462D
:1096D0000122054801F01EFA044B187008B1012060
:1096E00008BD0020FCE700BFB01600209402002057
:1096F00008B501460122002001F00CFA034B187056
:1097000008B1012008BD0020FCE700BF9402002042
:10971000F8B504460D461646104901F0ECFE104B14
:10972000187008B1C0B2F8BD022221460D4801F000
:1097300021FA0B4B187008B1C0B2F4E7094F0A4B7D
:1097400032462946384601F01AFC054C207038464E
:1097500001F069FD2070C0B2E5E700BF6806002097
:109760009402002080060020600600202DE9F041D0
:1097700004460F4690461D46434901F0BCFE434B4C
:109780001870E8B901222146414801F0F3F9064674
:109790003E4B187018BB29463D4801F059FD3B4B24
:1097A000187058B36420F7F79DFA054622463949E8
:1097B000F6F788FD2846F7F79DFA344B18780CE049
:1097C0006420F7F78FFA054622463349F6F77AFD0B
:1097D0002846F7F78FFA2D4B1878BDE8F081642002
:1097E000F7F780FA0546234632462C49F6F76AFD1C
:1097F0002846F7F77FFA254B1878EEE7284B4246C4
:109800003946234801F0CFFA0646204B187008BBB2
:1098100055B91F4BDA68234B1A603A705A787A7040
:109820009A78BA70DB78FB70194801F0FCFC0546A9
:10983000164B1870D8B16420F7F754FA0646234641
:109840002A461949F6F73EFD3046F7F753FA0F4B13
:109850001878C2E76420F7F745FA054623463246F2
:109860001249F6F72FFD2846F7F744FAEFE7642090
:10987000F7F738FA054622460D49F6F723FD284644
:10988000F7F738FAE3E700BF6806002094020020EB
:109890008006002000BE000844BD000868BD000826
:1098A0006406002088020020B8BD000890BD0008B2
:1098B000E0BD000810B504460C4901F01CFE0C4B3D
:1098C000187008B9C0B210BD0B222146094801F03A
:1098D00051F9074B187008B1C0B2F4E7054801F020
:1098E000A2FC034B1870C0B2EDE700BF6806002071
:1098F000940200208006002070B504461A4901F049
:10990000FAFD1A4B1870A0B9204601F016FE054664
:10991000164B1870D8B96420F7F7E4F905462246CB
:109920001349F6F7CFFC2846F7F7E4F90F4B187800
:1099300070BD6420F7F7D6F9054622460D49F6F7C3
:10994000C1FC2846F7F7D6F9084B1878F0E76420F1
:10995000F7F7C8F9064623462A460749F6F7B2FC48
:109960003046F7F7C7F9E1E76806002094020020C7
:1099700048BE000828BE00086CBE0008F8B50446C2
:109980000D461646104901F0B6FD104B187008B18F
:10999000C0B2F8BD322221460D4801F0EBF80B4B66
:1099A000187008B1C0B2F4E7094F0A4B3246294695
:1099B000384601F0E4FA054C2070384601F033FCDB
:1099C0002070C0B2E5E700BF6806002094020020C6
:1099D000800600206006002008B5044B03EB8002DF
:1099E000526852680344187A904708BD0C2700203B
:1099F00008B5084B1B5C53B9064B01221A5403EB04
:109A00008002526812680344187A904708BD00200B
:109A1000FCE700BF0C27002038B5044C04EB8005A0
:109A20006D68AD680444207AA84738BD0C27002033
:109A300038B5044C04EB80056D68ED680444207A69
:109A4000A84738BD0C27002010B5044B03EB800459
:109A5000646824690344187AA04710BD0C270020CD
:109A60004278007840EA02207047C378827842EA60
:109A70000322437843EA0223007840EA0320704738
:109A80000170090A417070470170C1F307234370E8
:109A9000C1F307438370090EC1707047944632B119
:109AA0000A78013102700130BCF1010CF8D1704725
:109AB00001700130013AFBD1704784469CF80000E8
:109AC0000CF1010C0B780131C01A013A01D00028C9
:109AD000F4D07047034600E00133187808B188429B
:109AE000FAD1704710B44FF0000C634602E04FF01B
:109AF000010C0133012B15D81A01184CA258002A69
:109B0000F5D00468A242F4D1144A02EB031254685F
:109B100082689442EDD1114A02EB031294684269C3
:109B20009442E6D1022B0BD0B1B90C4A02EB0313DD
:109B30009B89B3F5807F0DD000205DF8044B704702
:109B4000022914BF63464CF001030BB10020F4E777
:109B50001220F2E71020F0E71020EEE7E4260020C4
:109B6000002000E00130012804D80301034AD35843
:109B7000002BF7D1023818BF01207047E4260020DF
:109B800070B4002300E00133012B13D81A01234CD9
:109B9000A45802689442F6D1204A02EB031254689A
:109BA00082689442EFD11D4A02EB03129468426925
:109BB0009442E8D1022B08D0F9B1184A02EB031203
:109BC00092894ABB4FF480721DE00023012B05D817
:109BD0001A01124CA2580AB10133F7E7022B19D02F
:109BE0000E4D1C0105EB031206682E51846854606B
:109BF0004069906000209081DEE7084A02EB031282
:109C00009289013292B2054901EB03118A81581CF5
:109C100070BC70470020FBE70020F9E7E426002035
:109C20000138012815D80D4B03EB00139B89B3F5C0
:109C3000807F03D043B1013B9BB200E00023074A81
:109C400002EB0012938133B903010020034AD05084
:109C50007047022070470020704700BFE4260020B4
:109C6000002303E05DF8044B70470133012B11D84A
:109C70001A0109498A588242F7D110B41A01002406
:109C80008C500133012BEDD81A0103498A588242C6
:109C9000F7D1F3E7704700BFE4260020023983695B
:109CA000023B8B4204D94389C06A01FB0300704721
:109CB000002070470268C36A04339089B1FBF0F159
:109CC0005289B1FBF2F101E0091A0833186818B1A2
:109CD0008142F9D258680844704770B506460D466F
:109CE00001F11A00FFF7BCFE3378032B00D070BDE2
:109CF000044605F11400FFF7B3FE44EA0040F6E71E
:109D000070B506460C46154691B204F11A00FFF7ED
:109D1000B7FE3378032B00D070BD290C04F114007A
:109D2000FFF7AEFEF8E738B500234B72C36973B393
:109D300005460C460022134606E0BCF1090F0FD081
:109D4000A1184B72013263460A2B0ED803F1010CA5
:109D5000296ACB5C202BF6D0052BEED1E523ECE76E
:109D6000A1182E2048720132EAE7224400235372E0
:109D70002B6ADB7A2372286A1C30FFF776FE20609C
:109D8000286A1630FFF771FEE080000CA08038BD15
:109D90002DE9F84F81468A46D1F8008000F1240B66
:109DA0000B2220215846FFF783FE00252B4608276B
:109DB00029E0013618F806302F2BFAD05C2BF8D0AA
:109DC0004644CAF80060002D44D099F82430E52BB1
:109DD00035D0202C37D8042389F82F30002035E0E7
:109DE00014F0800F27D121461B48FFF773FE78BB84
:109DF000A4F16103DBB2192B01D8203CE4B20BF8CB
:109E00000540013533465E1C18F80340202CD7D995
:109E10005C2C18BF2F2CCDD02E2C18BFAF42DFD812
:109E20002E3C18BF01240B2F08BF44F0010464B975
:109E300008250B27E6E7803C084B1C5DD3E705238C
:109E400089F82430C5E70023C6E70620BDE8F88F6F
:109E50000620FBE70620F9E78CBE000890C000084A
:109E60000146006808B1024603E04FF0FF3070473A
:109E700001321378202B01D93A2BF9D13A2B01D09A
:109E800000207047034613F8010B3038092898BFAB
:109E90009A4203D128B901320A6070474FF0FF306F
:109EA00070474FF0FF30704738B50D46044698B103
:109EB00003689BB11A78A2B18188DA88914203D0F5
:109EC000092000242C6038BD5878FFF785FD10F07C
:109ED000010009D12468F5E70920F3E71C460920B1
:109EE000F0E709200024EDE709200024EAE72DE946
:109EF000F041C57815B92846BDE8F0810446076BE6
:109F000000F1340801233A4641464078FFF790FDBE
:109F10000546A0B90023E370636AFB1AE269934225
:109F2000E9D2A67808E0E3691F4401233A46414696
:109F30006078FFF77DFD013E012EF4D8DBE70125B7
:109F4000D9E770B5036B8B4202D10026304670BD55
:109F500004460D46FFF7CBFF06460028F6D1012345
:109F60002A4604F134016078FFF756FD10B101264E
:109F70004FF0FF352563E9E738B504460023C37089
:109F80004FF0FF330363FFF7DCFF30BB054604F2FD
:109F90003220FFF765FD4AF6552398421FD194F809
:109FA0003430E92B07D0636B03F0FF130D4A934263
:109FB00001D0022514E004F16A00FFF756FD20F0FD
:109FC0007F40094B98420BD004F18600FFF74DFD0E
:109FD000064B984204D0022502E0042500E0032548
:109FE000284638BDEB0090004641540046415433AA
:109FF0002DE9F04F87B00D46164600230B60FFF7A2
:10A000002FFF071EC0F26781BE4B53F82740002C7C
:10A0100000F066812C6006F0FE06237873B160784C
:10A02000FFF7DAFC10F0010508D1002E00F0548192
:10A0300010F0040F00F050810A254DE10023237039
:10A04000F8B26070FFF7D4FC10F0010F40F04A81C5
:10A050001EB110F0040F40F0478104F10C02022100
:10A060006078FFF7F1FC0546002840F03F81A289A7
:10A07000A2F500739BB2B3F5606F00F23981531EF5
:10A080001A4201D0012527E100212046FFF774FF85
:10A09000022800F088800026042800F02B81012887
:10A0A00000F22A8104F13F00FFF7DAFCB4F80C80DB
:10A0B000404540F0238104F14A00FFF7D1FC0746F8
:10A0C00020B904F15800FFF7D0FC0746E76194F887
:10A0D0004420A270531EDBB2012B00F2118107FB5A
:10A0E00002F3009394F84190A4F80A90B9F1000F9C
:10A0F00000F0108109F1FF3319EA030F40F00C81E1
:10A1000004F14500FFF7ACFC824620814FEA581B62
:10A11000B0FBFBF30BFB13039BB2002B40F0FE8064
:10A1200004F14700FFF79CFC019020B904F15400B2
:10A13000FFF79BFC019004F14200FFF791FC014600
:10A14000002800F0ED80009BC318BAFBFBFB5B44CA
:10A15000019A9A42C0F0E680D21AB2FBF9F04A4561
:10A16000C0F0E2804FF6F572904234D840F6F572B6
:10A1700090426AD94FF0020B2FE0002006AB03EBB0
:10A18000860343F8100C0136032E0ED804F1340078
:10A19000330103F5DF7318440379002BEDD0083049
:10A1A000FFF763FCEAE70026EEE700270AE0314606
:10A1B0002046FFF7E1FE01287FF66EAF0137032F3F
:10A1C0003FF66AAF06AB03EB870353F8106C002E23
:10A1D000EDD10320F2E74FF0030B00F10209C4F8C0
:10A1E000189026628A1962623344E362BBF1030F5E
:10A1F0002ED0BAF1000F00F09D80009B1A44A2629D
:10A20000BBF1020F35D009EB490209F0010303EB62
:10A2100052034344013BB3FBF8F3BB4200F28C8092
:10A220004FF0FF336361236180232371BBF1030F80
:10A2300022D084F800B0344A138801339BB21380D3
:10A24000E3802046FFF70CFD46E04FF0010BC4E72A
:10A2500004F15E00FFF704FC002867D1BAF1000F9B
:10A2600066D104F16000FFF700FCA0624FEA8903A9
:10A27000CFE74FEA4903CCE704F16400FFF7F0FBB6
:10A280000128D6D1711C2046FFF75BFE0028D0D1F3
:10A290000023237104F23220FFF7E2FB4AF6552334
:10A2A0009842C6D104F13400FFF7DFFB174B984208
:10A2B000BFD104F50670FFF7D8FB154B9842B8D113
:10A2C00004F50770FFF7D1FB606104F50870FFF734
:10A2D000CCFB2061ADE70B25284607B0BDE8F08F29
:10A2E0000C25F9E70325F7E70A25F5E70125F3E74C
:10A2F0000125F1E70125EFE70D25EDE70D25EBE75A
:10A300000D25E9E70827002004270020525261416B
:10A31000727241610D25DFE70D25DDE70D25DBE7D5
:10A320000D25D9E70D25D7E70D25D5E70D25D3E771
:10A330000D25D1E70D25CFE70D25CDE72DE9F04718
:10A34000012940F28E8004460D46174683698B42F0
:10A3500040F28B800378022B49D0032B60D0012B75
:10A3600040F0858001EB5108416A8389B8FBF3F323
:10A370001944FFF7E6FD0646002873D104F1340ABC
:10A3800008F10109A389B8FBF3F203FB128815F069
:10A39000010522D01AF8083003F00F0343EA07132F
:10A3A000DBB20AF808300123E370616AA389B9FBC4
:10A3B000F3F319442046FFF7C4FD0646002851D1A7
:10A3C000A389B9FBF3F203FB129945B1C7F3071355
:10A3D0000AF809300123E37044E0FBB2E1E71AF820
:10A3E0000930C7F3032223F00F031343F0E7416A58
:10A3F00083895B08B5FBF3F31944FFF7A2FD06461A
:10A4000080BB04F134006D00A389B5FBF3F203FBBC
:10A410001255B9B22844FFF733FB0123E37021E062
:10A42000416A83899B08B5FBF3F31944FFF789FD63
:10A430000646B8B927F0704704F13403AD00A2898D
:10A44000B5FBF2F102FB11551D442846FFF70DFB49
:10A4500000F0704139432846FFF716FB0123E370F3
:10A4600000E002263046BDE8F0870226FAE7022621
:10A47000F8E7F8B5056801296AD90C46AB698B4243
:10A4800068D92B78022B35D0032B49D0012B63D10F
:10A4900001EB5106696AAB89B6FBF3F31944284610
:10A4A000FFF74FFD10B14FF0FF3052E0771CAB8942
:10A4B000B6FBF3F203FB12662E4496F83460696A29
:10A4C000B7FBF3F319442846FFF73BFD002845D1BD
:10A4D000AB89B7FBF3F203FB12772F4497F83430C4
:10A4E00046EA032014F0010F01D0000931E0C0F367
:10A4F0000B002EE0696AAB895B08B4FBF3F31944E7
:10A500002846FFF71EFD60BB05F134006400AB89EF
:10A51000B4FBF3F203FB12442044FFF7A1FA18E066
:10A52000696AAB899B08B4FBF3F319442846FFF72B
:10A5300008FDC8B905F13400A400AB89B4FBF3F2FF
:10A5400003FB12442044FFF790FA20F0704000E033
:10A550000120F8BD0120FCE70120FAE74FF0FF30B1
:10A56000F7E74FF0FF30F4E74FF0FF30F1E72DE968
:10A57000F041D0F80080B1F5001F49D207460E46E1
:10A5800011F01F0F47D1416184681CBB98F800305F
:10A59000022B01D9D8F82840E4B9B8F80830B3EB59
:10A5A000561F3AD9D8F82830FB61BC61FB69E3B388
:10A5B000B8F80C20B6FBF2F21344FB6108F1340347
:10A5C000B8F80C20B6FBF2F102FB11610B443B62C0
:10A5D00000201EE0B8F80A50B8F80C3003FB05F56F
:10A5E000AE420FD321463846FFF743FF0446B0F191
:10A5F000FF3F14D0012814D9D8F81830834212D95B
:10A60000761BEDE721464046FFF748FBF861CCE7B3
:10A610000220BDE8F0810220FBE70220F9E70120DB
:10A62000F7E70220F5E70220F3E70220F1E72DE942
:10A63000F041054606680F4651B9D6F81080B8F1CA
:10A64000000F12D0B369434511D84FF001080EE056
:10A65000FFF70FFF034601284CD9B0F1FF3F4ED062
:10A66000B26982424BD8B84601E04FF00108444637
:10A670000CE021462846FFF7FCFE034678B1B0F116
:10A68000FF3F18BF01283AD0444537D00134B369A1
:10A69000A342EED8B8F1010F2ED90224E9E74FF01A
:10A6A000FF3221463046FFF749FE0246B0FA80F0FD
:10A6B0004009002F08BF002070B9A2B93461726947
:10A6C000B369023B9A4201D8013A7261337943F08F
:10A6D00001033371234612E0224639463046FFF724
:10A6E0002DFE0246E9E7012A01D0012307E04FF0E1
:10A6F000FF3304E0012302E0002300E000231846BA
:10A70000BDE8F081F8B50C46056801292ED906464A
:10A710001146AB69A3422BD94AB14FF0FF3228460C
:10A72000FFF70CFE074610B123E0A24221D92746CD
:10A7300021463046FFF79DFE0446E0B101281CD0BB
:10A74000B0F1FF3F1BD0002239462846FFF7F6FD47
:10A75000074670B96B69AA69911E8B42E5D2013335
:10A760006B612B7943F001032B71DEE7022700E0D8
:10A7700002273846F8BD0027FBE70227F9E7012743
:10A78000F7E738B504460568C1692846FFF7D9FBE5
:10A7900020B9236AE5221A700123EB7038BD2DE938
:10A7A000F84306684469C369002B74D005460F4618
:10A7B0002034B4F5001F70D2B189B4FBF1F201FB73
:10A7C00012423AB90133C3618169A1B93389B3EB4C
:10A7D000541F0CD96C6106F13403B289B4FBF2F159
:10A7E00002FB114423442B620020BDE8F8830023C0
:10A7F000C3610420F9E7B289B4FBF2F27389013B2B
:10A8000012EA0308E6D1FFF734FE8146012846D953
:10A81000B0F1FF3F45D0B369834234D88FB1A96905
:10A820002846FFF704FF814600283CD001283CD091
:10A83000B0F1FF3F3BD03046FFF759FB28B1012074
:10A84000D3E70023EB610420CFE7B289002106F1B2
:10A850003400FFF72DF949463046FFF71FFA306301
:10A86000738998450BD20123F3703046FFF73FFB05
:10A87000F8B908F10108336B01333363F0E7336B48
:10A88000A3EB08033363C5F8189049463046FFF739
:10A8900005FAE8619EE70420A7E70420A5E7022067
:10A8A000A3E70120A1E707209FE702209DE7012001
:10A8B0009BE7012099E770B5044606680021FFF781
:10A8C00056FE054640B1284670BD00212046FFF7E0
:10A8D00066FF05460028F6D1E1693046FFF731FBF7
:10A8E00005460028EFD1206A03787BB1C37A03F0D4
:10A8F0003F03A371C37A13F0080FE6D10B2204F1D2
:10A900002401FFF7DAF80028DFD1DCE70425DAE7D5
:10A9100030B583B004460191056801E0013301932D
:10A92000019B1A782F2AF9D05C2AF7D00022A26066
:10A930001B781F2B21D901A92046FFF729FA0346CE
:10A9400018BB2046FFF7B7FF94F82F200346F8B94D
:10A9500012F0040F19D1A37913F0100F1FD005F1D5
:10A9600034016369AA89B3FBF2F002FB1033194486
:10A970002846FFF7B2F9A060DDE7802384F82F3086
:10A9800011462046FFF7F3FD0346184603B030BDDD
:10A990000428FAD112F0040FF7D10523F5E70523B7
:10A9A000F3E7F8B504460E4607680021FFF7DFFD20
:10A9B0000246B8B9002506E0002501212046FFF730
:10A9C000EEFE024670B9E1693846FFF7BAFA024670
:10A9D00040B9236A1B78002B18BFE52BECD1013559
:10A9E000B542EAD1042A01D01046F8BD0722FBE7A0
:10A9F00070B5044606680121FFF7D3FF054608B18C
:10AA0000284670BDE1693046FFF79BFA05460028ED
:10AA1000F6D120220021206AFFF74AF80B2204F128
:10AA20002401206AFFF73AF80123F370E8E7F8B54C
:10AA300004460E460568042705E000212046FFF77E
:10AA4000AEFE0746E8B9E169D9B12846FFF779FAC1
:10AA50000746B0B9236A1A7892B1DB7A03F03F0354
:10AA6000A371E52A18BF2E2AE7D00F2BE5D023F0DB
:10AA70002003082B14BF00230123B342DDD100E0E3
:10AA800004270FB10023E3613846F8BD70B50446D2
:10AA9000FFF72DFA054648B92378032B08D000228A
:10AAA00011466078FEF7D0FF00B10125284670BD41
:10AAB0002379012BF3D104F13406A2890021304619
:10AAC000FEF7F6FF4AF6552104F23220FEF7D8FFD2
:10AAD0000E493046FEF7D8FF0D4904F50670FEF723
:10AAE000D3FF616904F50770FEF7CEFF216904F515
:10AAF0000870FEF7C9FF226A013222630123314642
:10AB00006078FEF795FF00232371C8E75252614138
:10AB10007272416170B584B0019000911646039144
:10AB200003A8FFF79DF9041E20DB114B53F82450B6
:10AB300025B12846FFF794F800232B70019B0BB139
:10AB400000221A70019B0A4A42F82430721E18BF74
:10AB50000122002B08BF42F0010212B1002004B014
:10AB600070BD01A96846FFF743FAF8E70B20F6E746
:10AB7000082700202DE9F04391B00191002800F052
:10AB800010811446064602F03F073A4603A901A881
:10AB9000FFF72EFA054628B100233360284611B08E
:10ABA000BDE8F083039B0493019904A8FFF7B0FE6E
:10ABB000054660B99DF93F30002B52DB14F03E0F83
:10ABC00014BF0121002104A8FEF78CFF054614F0F4
:10ABD0001C0F5CD0002D50D0042D44D047F0080746
:10ABE000002DD9D117F0080F61D0FAF749F80446C3
:10ABF00001460C980E30FEF747FF21460C981630A0
:10AC0000FEF742FF0C9B2022DA72DDF80C80DDF8A3
:10AC1000309049464046FFF760F804460022494616
:10AC20004046FFF76DF800210C981C30FEF72CFF12
:10AC3000039B0122DA70002C39D0039BD3F83080BB
:10AC40000022214604A8FFF75DFD05460028A3D198
:10AC500041460398FFF775F90546013C039B1C61CB
:10AC600025E00625B3E7FEF77BFF08B91225B5E717
:10AC700004A8FFF7BDFE0546B0E79DF8163013F0B7
:10AC8000110F13D114F0040FAAD0082584E7002D6A
:10AC900082D19DF8163013F0100F7ED114F0020F00
:10ACA00005D013F0010F02D0072575E70725002D09
:10ACB0007FF472AF17F0080F01D047F04007039BF5
:10ACC0001B6B73620C9BB362012F94BF00210121A7
:10ACD00004A8FEF755FF306108B902255CE7039C24
:10ACE000DDF8308041462046FEF7F7FFB06008F1FE
:10ACF0001C00FEF7BAFEF0600021F1623460E388C8
:10AD0000B380377571753162B16106F130084FF467
:10AD100080524046FEF7CCFE17F0200F39D0F46881
:10AD2000002C36D0B461039B5F899B8903FB07F736
:10AD3000B16801E00225E41BBC4294BF002301235B
:10AD40005DB953B13046FFF794FB01460128F1D9B4
:10AD5000B0F1FF3FEFD10125EDE7F161002D7FF468
:10AD60001BAF039FB7F80C90B4FBF9F309FB134337
:10AD70007BB13846FEF792FF08B902250CE7B4FB19
:10AD8000F9F202443262012341467878FEF744FE2C
:10AD900028B9002D3FF402AFFEE60425FCE60125AC
:10ADA000FAE60925FAE62DE9F04F85B004460F468C
:10ADB000154698460023C8F8003003A9FFF774F839
:10ADC0000190002840F0B980637D0193002B40F092
:10ADD000B480237D13F0010F00F0CE80E668A369F4
:10ADE000F61AAE4267D32E4665E0E36A1BB12046F1
:10ADF000FEF760FF73E0E1692046FFF73AFB6EE083
:10AE00004FF0020A84F815A0CDF804A095E04FF0A9
:10AE1000010A84F815A0CDF804A08EE04FF0020AD4
:10AE200084F815A0CDF804A087E094F91430002B25
:10AE300004DB039B9D890AFB05F532E0236AA3EB43
:10AE400009035345F5D2039A928904F1300102FBBC
:10AE50000370FEF723FEECE7226A4A450DD094F911
:10AE60001430002B6DDB01234A4604F130010398B6
:10AE70004078FEF7D1FD002877D1C4F82090039BDD
:10AE80009D89A369B3FBF5F205FB1233ED1AAE42BF
:10AE900000D2354604F130012A4619443846FEF7FF
:10AEA000FDFD2F44A3692B44A361D8F800302B4447
:10AEB000C8F80030761B002E3FD0A169039A95890F
:10AEC000B1FBF5F305FB1313002BD8D1B1FBF5F55E
:10AED0005389013B1D4008D1002986D1A068012873
:10AEE0008ED9B0F1FF3F92D0E061DDF80CB0E1699E
:10AEF0005846FEF7D3FE814600288FD0A944BBF800
:10AF00000C30B6FBF3FAB342A6D805EB0A03BBF844
:10AF10000A20934201D9A2EB050A53464A46394614
:10AF20009BF80100FEF778FD00283FF47EAF4FF05C
:10AF3000010A84F815A0CDF804A0019805B0BDE879
:10AF4000F08F012304F130019BF80100FEF770FD42
:10AF500020B9237D03F07F03237584E74FF0010AB6
:10AF600084F815A0CDF804A0E7E74FF0010A84F8B3
:10AF700015A0CDF804A0E0E707230193DDE72DE954
:10AF8000F04F85B004460F46154698460023C8F892
:10AF9000003003A9FEF788FF019000284AD1637DA5
:10AFA0000193002B46D1237D13F0020F00F0EC80BB
:10AFB000A369EB42C0F0B680DD43B3E0E36A002B47
:10AFC0003CD02046FEF776FE002800F0D88001280D
:10AFD00039D0B0F1FF3F3DD0E061A36803B9A06074
:10AFE00094F91430002B3CDBDDF80CB0E1695846D5
:10AFF000FEF754FE8146002848D0B144BBF80C301F
:10B00000B5FBF3FAAB425FD806EB0A03BBF80A20A4
:10B01000934201D9A2EB060A53464A4639469BF8A9
:10B020000100FEF705FDC0B34FF0010A84F815A03A
:10B03000CDF804A0019805B0BDE8F08FE169204685
:10B04000FFF7F5FAC0E74FF0020A84F815A0CDF833
:10B0500004A0EFE74FF0010A84F815A0CDF804A092
:10B06000E8E70123226A04F1300103984078FEF7F3
:10B07000DFFC20B9237D03F07F032375B4E74FF095
:10B08000010A84F815A0CDF804A0D3E74FF0020A16
:10B0900084F815A0CDF804A0CCE7236AA3EB09033C
:10B0A000534504D3039B9E890AFB06F62BE0039AC3
:10B0B000928902FB037104F13000FEF7EFFC237D5F
:10B0C00003F07F032375EDE7236A4B4503D0A269A4
:10B0D000E3689A4242D3C4F82090039B9E89A369F7
:10B0E000B3FBF6F206FB1233F61AB54200D22E4637
:10B0F00004F13000324639461844FEF7CFFC237D78
:10B1000063F07F0323753744A3693344A361E26886
:10B11000934238BF1346E360D8F800303344C8F890
:10B120000030AD1B5DB3A169039A9689B1FBF6F3BC
:10B1300006FB1313002BD0D1B1FBF6F65389013B6C
:10B140001E407FF44DAF00297FF438AFA06800287F
:10B150007FF43DAF2046FFF76AFA35E701234A4600
:10B1600004F130019BF80100FEF756FC0028B2D034
:10B170004FF0010A84F815A0CDF804A05AE7237D0A
:10B1800043F04003237555E70723019352E770B559
:10B1900082B0044601A9FEF787FE70B9237D13F043
:10B1A000400F0AD013F0800F09D1F9F769FD054669
:10B1B000616A0198FEF7C5FE78B102B070BD012347
:10B1C000226A04F1300101984078FEF731FC40BB5F
:10B1D000237D03F07F032375E7E7A66AF37A43F044
:10B1E0002003F372A26831462068FEF789FDE1680A
:10B1F00006F11C00FEF748FC294606F11600FEF792
:10B2000043FC002106F11200FEF73AFC019B0122EB
:10B21000DA700198FFF73AFC237D23F04003237591
:10B22000CBE70120C9E710B582B00446FFF7AFFFB6
:10B2300008B102B010BD01A92046FEF735FE002876
:10B24000F7D12069FEF7ECFC0028F2D12060F0E78E
:10B250002DE9F04F83B004460D4601A9FEF724FE08
:10B26000064678B9667D6EB9E36A002B00F08E80E1
:10B27000B5F1FF3F0AD0E768AF4200D32F46A76180
:10B28000002F3FD1304603B0BDE8F08F984658F804
:10B2900004BBD4F808A0BAF1000F27D04FF0020980
:10B2A00009F102095146002701370D462046FFF7F4
:10B2B000E0F80146012813D9B0F1FF3F13D0013562
:10B2C0008542F1D0CB4505D3434643F8087BC8F807
:10B2D00004A09846019B9B698B4209D98A46DFE707
:10B2E00002266675CEE701266675CBE74FF00209A8
:10B2F000E36AC3F80090D94500F2FB800023C8F848
:10B300000030BFE77D1E29462046FEF7D3FC0146EC
:10B31000E061DDF804804046FEF7C0FC00B3B8F8F9
:10B320000C30B5FBF3F5B8F80A20013A1540054496
:10B33000B7FBF3F203FB1277002FA3D0226AAA42D5
:10B34000A0D094F91430002B0DDB01232A4604F120
:10B35000300101984078FEF75FFBA0B9256291E7C4
:10B36000022666758EE7012304F1300198F801008A
:10B37000FEF75EFB20B9237D03F07F032375E4E72E
:10B38000012666757EE7012666757BE7E368AB42BA
:10B3900004D2227D12F0020F00D11D46A3690022C3
:10B3A000A261E5B1019AB2F80A80928902FB08F81D
:10B3B00073B16A1EB2FBF8F2013BB3FBF8F18A42AB
:10B3C00006D3C8F100021340A361EF1AE56904E057
:10B3D000A06850B3E0612F460546002D45D1A36912
:10B3E000E268934204D9E360227D42F04002227574
:10B3F00001988289B3FBF2F102FB1133002B3FF479
:10B4000041AF226AAA423FF43DAF94F91430002BB9
:10B410005DDB01232A4604F1300101984078FEF7F4
:10B42000FBFA002862D125622CE700212046FFF7B5
:10B43000FEF8012804D0B0F1FF3F04D0A060C9E7B6
:10B44000022666751EE7012666751BE7294620461B
:10B45000FFF70FF80546B5F1FF3F2DD0012D2ED98E
:10B46000019B9B69AB422AD9E561474510D9A7EBFF
:10B470000807A3694344A361237D13F0020FE5D0BD
:10B4800029462046FFF7D3F805460028E3D10746B2
:10B49000A3693B44A3610198B0F80C80B7FBF8F3B3
:10B4A00008FB13738BB12946FEF7F8FB054648B13C
:10B4B000B7FBF8F73D4492E701266675E2E60226FF
:10B4C0006675DFE602266675DCE61D4687E7012322
:10B4D00004F130014078FEF7ABFA20B9237D03F088
:10B4E0007F03237595E701266675CBE60126667511
:10B4F000C8E61126C6E630B58FB001900C46002292
:10B5000002A901A8FEF774FD054610B128460FB048
:10B5100030BD019902A8FFF7FBF905460028F5D1D7
:10B520009DF93730002B06DB002CEFD0214602A816
:10B53000FEF7F9FBEAE70625E8E7F0B59DB00190D4
:10B54000022203A901A8FEF753FD039B10930446B2
:10B5500010B120461DB0F0BD019910A8FFF7D8F931
:10B5600004460028F5D1022110A8FEF7BBFA0446D4
:10B570000028EED19DF96F30002B3CDB9DF8465042
:10B5800015F0010F39D1039F18993846FEF7A5FB36
:10B59000064615F0100F13D1002CDAD110A8FFF7D2
:10B5A000F0F80446B0FA80F04009002E08BF0020F1
:10B5B000D0B9002CCDD10398FFF768FA0446C8E74C
:10B5C00004970690002104A8FEF7D1FF0446002846
:10B5D000BFD1002104A8FFF72AFA044610B10428BD
:10B5E000DAD1DBE70724D7E70022314610A8FFF7BE
:10B5F00089F80446DDE70624ABE70724A9E7000045
:10B60000134B5B7A13BB10B5044603F0FF00104BDD
:10B6100093F809C05FFA8CFC4FF0000E03F80CE0C1
:10B6200093F809C003EB8C0CCCF804405C7A1C4402
:10B6300022725A7A541CE4B25C7230320A703A2395
:10B640004B702F238B7081F803E010BD01207047F1
:10B650000C27002008B50022FFF7D2FF08BD00002C
:10B6600010B503460C4A0D490D48006840B10C481E
:10B6700000680344521A934206D8094A136010BD69
:10B680000748084C0460F2E7F5F7B8F80C230360AC
:10B690004FF0FF30F3E700BF00000820004000003B
:10B6A0001827002020270020026852E8003F23F4DA
:10B6B000907342E800310029F6D1026802F10803D4
:10B6C00053E8003F23F00103083242E8003100292B
:10B6D000F3D1036E012B06D02023C0F88030002365
:10B6E000036683667047026852E8003F23F0100348
:10B6F00042E800310029F6D1EEE7000010B504461B
:10B7000083680269134342691343C26913430168A2
:10B710000868914A02401A430A602268536823F479
:10B720004053E1680B435360A269236A1A432168BE
:10B730008B6823F4306313438B602368874A9342FA
:10B7400018D0874A93423AD0864A93424FD0864ACD
:10B7500093425ED0854A93426DD0854A93427FD012
:10B76000844A934200F09180834A934200F0A28081
:10B7700010230BE0814BD3F8903003F00303032B2D
:10B780001BD8DFE803F00216AB180123E069B0F51F
:10B79000004F00F0D780082B00F23881DFE813F06B
:10B7A00014012701120136012A0136013601360142
:10B7B0002D010423EAE70823E8E71023E6E76F4BAF
:10B7C000D3F8903003F00C030C2B0ED8DFE803F015
:10B7D000070D0D0D090D0D0D880D0D0D0B0000232E
:10B7E000D4E70423D2E70823D0E71023CEE7634B46
:10B7F000D3F8903003F03003202B73D005D8002B02
:10B8000072D0102B72D10423C0E7302B70D10823E3
:10B81000BCE75A4BD3F8903003F0C003802B69D0BB
:10B8200005D8002B68D0402B68D10423AEE7C02B8D
:10B8300066D10823AAE7514BD3F8903003F4407344
:10B84000B3F5007F5ED006D8002B5DD0B3F5807FC6
:10B850005CD104239AE7B3F5407F59D1082395E7DB
:10B86000464BD3F8903003F44063B3F5006F51D0EA
:10B8700006D8002B50D0B3F5806F4FD1042385E755
:10B88000B3F5406F4CD1082380E73C4BD3F89030A0
:10B8900003F44053B3F5005F44D006D8002B43D0E7
:10B8A000B3F5805F42D1042370E7B3F5405F3FD129
:10B8B00008236BE7314BD3F8903003F44043B3F5E2
:10B8C000004F37D005D8BBB3B3F5804F36D1042332
:10B8D0005CE7B3F5404F33D1082357E7022355E720
:10B8E000022353E7022351E700234FE710234DE7DC
:10B8F00010234BE7022349E7002347E7102345E7DE
:10B90000102343E7022341E700233FE710233DE7ED
:10B9100010233BE7022339E7012337E7102335E7FC
:10B92000102333E7022331E700232FE710232DE70D
:10B9300010232BE7022329E7002327E7102325E71D
:10B94000102323E7082B5BD8DFE803F01A343A5AB8
:10B95000375A5A5A1E0000BFF369FFEF001001402A
:10B960000044004000480040004C004000500040AF
:10B970000014014000780040007C00400038024084
:10B98000FAF7D2FD00283DD06268530803EB40036C
:10B99000B3FBF2F3A3F110014FF6EF72914233D8EB
:10B9A0009AB222F00F02C3F3420313432268D3601A
:10B9B000002030E0FAF7C8FDE4E7FAF7A5FCE1E77C
:10B9C0001748E1E7164802E0FAF7AEFD00B36368F6
:10B9D00000EB5300B0FBF3F0A0F110024FF6EF7351
:10B9E0009A4217D8236880B2D860002013E0FAF793
:10B9F000ABFDEBE7FAF788FCE8E74FF40040E6E739
:10BA0000012008E0002006E0012004E0012002E01F
:10BA1000002000E001200023A366E36610BD00BF04
:10BA20000024F400436A13F0080F06D0026853683C
:10BA300023F40043416B0B435360436A13F0010F3F
:10BA400006D00268536823F40033816A0B435360C5
:10BA5000436A13F0020F06D00268536823F4803360
:10BA6000C16A0B435360436A13F0040F06D00268A7
:10BA7000536823F48023016B0B435360436A13F034
:10BA8000100F06D00268936823F48053816B0B4338
:10BA90009360436A13F0200F06D00268936823F482
:10BAA0000053C16B0B439360436A13F0400F0AD0FD
:10BAB0000268536823F48013016C0B435360036CDA
:10BAC000B3F5801F0BD0436A13F0800F06D00268D5
:10BAD000536823F40023816C0B4353607047026862
:10BAE000536823F4C003416C0B435360EBE72DE92B
:10BAF000F84305460E4617469946DDF820802B6828
:10BB0000DC6936EA04040CBF01240024BC423AD1AB
:10BB1000B8F1FF3FF3D0FBF731FAA0EB0900404545
:10BB200034D8B8F1000F33D02B681A6812F0040F24
:10BB3000E5D0B6F1400218BF0122802EDFD0002AE6
:10BB4000DDD0DA6912F0080F11D1DA6912F4006F52
:10BB5000D5D04FF400621A622846FFF7A5FD2023D6
:10BB6000C5F88430002385F8783003200CE00824E1
:10BB70001C622846FFF798FDC5F88440002385F82D
:10BB80007830012000E00020BDE8F8830320FBE7C7
:10BB90000320F9E730B583B004460023C0F88430B1
:10BBA000FBF7ECF905462268126812F0080F0FD176
:10BBB00023681B6813F0040F26D12023E367C4F821
:10BBC000803000202066606684F8780003B030BDC5
:10BBD0006FF07E430093034600224FF4001120468D
:10BBE000FFF785FF0028E3D0226852E8003F23F0EA
:10BBF000800342E800310029F6D12023E3670023C7
:10BC000084F878300320E1E76FF07E4300932B4601
:10BC100000224FF480012046FFF769FF0028CCD0B6
:10BC2000226852E8003F23F4907342E80031002973
:10BC3000F6D1226802F1080353E8003F23F0010324
:10BC4000083242E800310029F3D12023C4F88030C3
:10BC5000002384F878300320B8E768B310B50446B1
:10BC6000C36F03B32423E3672268136823F001033F
:10BC70001360636AE3B92046FFF740FD012811D045
:10BC80002268536823F4904353602268936823F03A
:10BC90002A0393602268136843F00103136020466F
:10BCA000FFF778FF10BD80F87830F9F751FDD9E73C
:10BCB0002046FFF7B7FEDEE701207047DFF834D0FB
:10BCC000FDF7FAFC0C480D490D4A002302E0D45858
:10BCD000C4500433C4188C42F9D30A4A0A4C0023D6
:10BCE00001E013600432A242FBD3F4F70DFDF8F734
:10BCF00021F8704700000820000000205C000020B0
:10BD000020C100085C0000201C270020FEE7000086
:10BD1000F8B500BFF8BC08BC9E467047F8B500BF38
:08BD2000F8BC08BC9E46704708
:10BD28002F000000434F4D4D414E442E54585400AF
:10BD380046494C45312E5458540000004552525241
:10BD48004F52212121202A25732A20646F657320F0
:10BD58006E6F74206578697374730A0A00000000B6
:10BD68004552524F52212121204E6F2E202564200A
:10BD7800696E206F70656E696E672066696C6520F4
:10BD88002A25732A0A0A00004552524F52212121BE
:10BD9800204E6F2E20256420696E207265616469CB
:10BDA8006E672066696C65202A25732A0A0A0000D6
:10BDB8004552524F52212121204E6F2E20256420BA
:10BDC800696E20636C6F73696E672066696C6520A5
:10BDD8002A25732A0A0A000046696C65202A2573F9
:10BDE8002A20434C4F53454420737563636573732E
:10BDF80066756C6C790A00004552524F5221212118
:10BE08002043616E2774207365656B207468652014
:10BE180066696C653A2020202A25732A0A0A0000E0
:10BE28004552524F52212121202A25732A20646F1E
:10BE38006573206E6F74206578697374730A0A00DD
:10BE48002A25732A20686173206265656E207265F1
:10BE58006D6F766564207375636365737366756C5F
:10BE68006C790A004552524F52204E6F2E2025649D
:10BE780020696E2072656D6F76696E67202A25735A
:10BE88002A0A0A00222A2B2C3A3B3C3D3E3F5B5DA6
:10BE98007C7F0000232D302B20000000686C4C00B4
:10BEA80065666745464700003031323334353637EA
:10BEB80038394142434445460000000030313233AE
:10BEC80034353637383961626364656600000000CE
:10BED8000000000E0000000000000000000000400C
:10BEE8000000000000000000001F0000000000002B
:10BEF8000E000000000000000000000030301101BA
:10BF0800FFFF000001010300000000000000000026
:10BF180000000000000000000040000000020000D7
:10BF28000000000000000000000000000000000009
:10BF380000000000000000000000000000000000F9
:10BF48000000000000000000A00F0000F03F00010A
:10BF580001000100000000000000000000000000D7
:10BF6800000000400000000000000000001F00006A
:10BF7800000000000E0000000000000000000000AB
:10BF880012322101FFFF0000010103000000000040
:10BF98000000000000000000000000000040000059
:10BFA80006069919009A0000000000000000000031
:10BFB80000000000A00F00000000000000000000CA
:10BFC8000000000000000000000000000000000069
:10BFD8000000FF160100010000000100020003003C
:10BFE8000400050006000700080009000A000B000D
:10BFF8000C000D000E001F0020002200230024006A
:10C00800250026002700280029002A002B002C00E4
:10C018002D002E002F003000310032003300340094
:10C028003500360037003E003F0040004100420026
:10C03800430044004500470050005100520053009F
:10C048005400550056005700580059005A005B002C
:10C058005C005D005E005F001E001D00954B00083F
:10C06800BD4B0008C54B0008E94B00080D4C000803
:10C0780000000000010203040000000000000000AE
:10C08800010203040607080943554541414141435C
:10C0980045454549494941414592924F4F4F55556C
:10C0A800594F554F9C4F9E9F41494F55A5A5A6A74F
:10C0B800A8A9AAABACADAEAFB0B1B2B3B4414141DF
:10C0C800B8B9BABBBCBDBEBFC0C1C2C3C4C541417B
:10C0D800C8C9CACBCCCDCECFD1D1454545494949B0
:10C0E80049D9DADBDCDD49DF4FE14F4F4F4FE6E856
:10C0F800E85555555959EEEFF0F1F2F3F4F5F6F726
:08C10800F8F9FAFBFCFDFEFF53
:08C11000004AFF7F010000005E
:04C1180069020008B0
:04C11C0041020008D4
:10C12000040000200000000080000020E800002043
:10C13000500100200000000000000000000000008E
:10C1400000000000000000000000000000000000EF
:10C1500000000000000000000000000000000000DF
:10C1600000000000000000000000000000000000CF
:0CC1700001010000100000000024F40099
:040000050800BCBD76
:00000001FF
